:100000000C942E060C944B060C944B060C944B0649
:100010000C944B060C944B060C944B060C944B061C
:100020000C944B060C944B060C944B060C944B060C
:100030000C944B060C944B060C94E30A0C944B0660
:100040000C944B060C9483070C9426070C94E8063A
:100050000C944B060C94DC170C944B060C944B063A
:100060000C944B060C944B06756E6974203C20531F
:1000700045525F434E5400626572746F732F637014
:10008000752F6176722F6472762F7365725F6D655E
:1000900067612E630073697A65203E2031006265D6
:1000A00072746F732F7374727563742F6669666FE1
:1000B0006275662E680066642D3E68772D3E727804
:1000C00062756666657200626572746F732F647222
:1000D000762F7365722E630066642D3E68772D3E21
:1000E000747862756666657200626572746F732FEC
:1000F0006472762F7365722E63002166642D3E69EB
:10010000735F6F70656E00626572746F732F6472D7
:10011000762F7365722E6300756E6974203C2063C0
:100120006F756E746F66287365725F68616E646C5C
:1001300065732900626572746F732F6472762F7312
:1001400065722E6300706F72742D3E69735F6F70FD
:10015000656E00626572746F732F6472762F7365BB
:10016000722E630066642D3E5F74797065203D3D9C
:10017000204B46545F53455249414C0062657274AE
:100180006F732F6472762F7365722E680021746905
:100190006D65725F696E697469616C697A65640026
:1001A000626572746F732F6472762F74696D6572F5
:1001B0002E63002674696D65722D3E6C696E6B004E
:1001C000626572746F732F6472762F74696D6572D5
:1001D0002E630066642D3E72656164006265727410
:1001E0006F732F696F2F6B66696C652E680066648C
:1001F0002D3E777269746500626572746F732F6942
:100200006F2F6B66696C652E68006275665F706F34
:10021000696E746572203E3D20627566006265728B
:10022000746F732F6D776172652F666F726D617475
:1002300077722E63006368616E6E656C0062657232
:10024000746F732F6E65742F617832352E6300637F
:10025000747800626572746F732F6E65742F6178A5
:1002600032352E63006973616C6E756D28632920C9
:100270007C7C2063203D3D2027202700626572742E
:100280006F732F6E65742F617832352E630063743F
:10029000782D3E6372635F6F7574203D3D20415839
:1002A00032355F4352435F434F52524543540062DD
:1002B0006572746F732F6E65742F617832352E639B
:1002C00000706174685F6C656E203E3D2032006294
:1002D0006572746F732F6E65742F617832352E637B
:1002E000007061746800626572746F732F6E65745C
:1002F0002F617832352E630066642D3E636C656134
:100300007265727200626572746F732F696F2F6B02
:1003100066696C652E680066642D3E6572726F7248
:1003200000626572746F732F696F2F6B66696C65FD
:100330002E68000000891112239B322446AD5736E7
:1003400065BF74488CC19D5AAFD3BE6CCAE5DB7ED5
:10035000E9F7F88110080193331A22A5562C47B704
:10036000753E64C99C408DDBBF52AEEDDA64CBFFB5
:10037000F976E802218B30100299132667AF7634A4
:1003800044BD554AADC3BC588ED19F6EEBE7FA7C95
:10039000C8F5D983310A2091121803A7772E66B5C4
:1003A000543C45CBBD42ACD99E508FEFFB66EAFD75
:1003B000D874C904428D5316619F702004A9153268
:1003C00027BB364CCEC5DF5EEDD7FC6888E1997A55
:1003D000ABF3BA85520C4397711E60A1142805B384
:1003E000373A26CDDE44CFDFFD56ECE9986089FB35
:1003F000BB72AA06638F7214409D512225AB343024
:1004000006B9174EEFC7FE5CCCD5DD6AA9E3B87814
:100410008AF19B87730E6295501C41A3352A24B143
:10042000163807CFFF46EEDDDC54CDEBB962A8F9F4
:100430009A708B088481951AA793B62CC2A5D33ED7
:10044000E1B7F04008C919522BDB3A644EED5F76F4
:100450006DFF7C899400859BB712A6ADD224C3BFE3
:10046000F136E0C1184809D33B5A2AE55E6C4FF7D4
:100470007D7E6C0AA583B4188691972EE3A7F23C83
:10048000C0B5D14229CB38500AD91B666FEF7E74B4
:100490004CFD5D8BB502A499961087AFF326E2BDA3
:1004A000D034C1C3394A28D11A580BE77F6E6EF594
:1004B0005C7C4D0CC685D71EE597F42880A1913A47
:1004C000A3B3B2444ACD5B5669DF78600CE91D7274
:1004D0002FFB3E8DD604C79FF516E4A9902081BB63
:1004E000B332A2C55A4C4BD7795E68E11C680DF354
:1004F0003F7A2E0EE787F61CC495D52AA1A3B03803
:1005000082B193466BCF7A5448DD59622DEB3C7033
:100510000EF91F8FF706E69DD414C5ABB122A0B922
:10052000923083C77B4E6AD5585C49E33D6A2CF113
:100530001E780F6368203C3D2035004D6F64656D6B
:100540002F68617264776172652E630066642D3E68
:100550005F74797065203D3D204B46545F414653A2
:100560004B004D6F64656D2F6166736B2E68008064
:100570008183848687898A8C8E8F919294959798AF
:100580009A9B9D9EA0A2A3A5A6A7A9AAACADAFB019
:10059000B2B3B5B6B7B9BABCBDBEC0C1C2C4C5C698
:1005A000C8C9CACBCDCECFD0D2D3D4D5D6D7D9DA3D
:1005B000DBDCDDDEDFE0E1E2E3E4E5E6E7E8E9EA13
:1005C000EAEBECEDEEEEEFF0F1F1F2F3F3F4F5F52A
:1005D000F6F6F7F8F8F9F9FAFAFAFBFBFCFCFCFD81
:1005E000FDFDFDFEFEFEFEFEFFFFFFFFFFFFFF54D1
:1005F00058205461696C3A2025640A0054582050F0
:100600007265616D626C653A2025640A0053796DEC
:10061000626F6C3A2025630A0053796D626F6C201B
:100620007461626C653A207374616E646172640A0D
:100630000053796D626F6C207461626C653A206161
:100640006C7465726E6174650A00446972656374E6
:1006500069766974793A2025640A004761696E3ABF
:100660002025640A004865696768743A2025640A91
:1006700000506F7765723A2025640A004175746FE7
:100680002D61636B206D657373616765733A204FED
:1006900066660A004175746F2D61636B206D65732A
:1006A00073616765733A204F6E0A00506174683257
:1006B0003A20252E36732D25640A00506174683166
:1006C0003A20252E36732D25640A0044657374691B
:1006D0006E6174696F6E3A20252E36732D25640A7B
:1006E0000043616C6C7369676E3A20252E36732D5A
:1006F00025640A00436F6E66696775726174696F7D
:100700006E3A0A00300A004572726F723A20496EE2
:1007100076616C696420636F6D6D616E640A00457B
:1007200072726F723A20496E76616C6964207661EC
:100730006C756520666F72205458207461696C0A6C
:10074000005458205461696C2073657420746F20C4
:1007500025646D730A004572726F723A20496E7695
:10076000616C69642076616C756520666F722070BB
:100770007265616D626C650A00507265616D626CD4
:10078000652073657420746F2025646D730A0031D1
:100790000A004D657373616765206175746F2D6123
:1007A000636B2064697361626C65640A00310A00DE
:1007B0004D657373616765206175746F2D61636B3F
:1007C00020656E61626C65640A00310A00526574CE
:1007D00072696564206C617374206D657373616701
:1007E000650A00310A000A002D25640A004D657370
:1007F0007361676520726563697069656E743A201C
:10080000252E367300310A000A002D25640A004D9A
:1008100065737361676520726563697069656E747D
:100820003A20252E367300310A0053656C656374D7
:100830006564207374616E646172642073796D62A3
:100840006F6C207461626C650A0053656C6563743B
:10085000656420616C7465726E6174652073796D76
:10086000626F6C207461626C650A0053796D626F0F
:100870006C2073657420746F2025630A00446972CC
:1008800065637469766974792073657420746F2068
:1008900025646465670A00446972656374697669F2
:1008A00074792073657420746F206F6D6E690A000F
:1008B000310A00310A004761696E20736574207443
:1008C0006F20256464420A00310A00416E74656E2F
:1008D0006E61206865696768742073657420746F41
:1008E00020256C646D204141540A00310A00506F8C
:1008F0007765722073657420746F202564770A0011
:10090000310A004C6F6E6774697475646520736595
:100910007420746F20252E39730A00310A004C614F
:100920007469747564652073657420746F20252E56
:1009300038730A00310A005072696E7420494E46BD
:100940004F2064697361626C65640A00310A00506B
:1009500072696E7420494E464F20656E61626C6507
:10096000640A00310A005072696E74204441544197
:100970002064697361626C65640A00310A00507218
:10098000696E74204441544120656E61626C6564F7
:100990000A00310A005072696E7420504154482098
:1009A00064697361626C65640A00310A005072699F
:1009B0006E74205041544820656E61626C65640A13
:1009C00000310A005072696E7420445354206469E7
:1009D0007361626C65640A00310A005072696E745A
:1009E0002044535420656E61626C65640A00310ACC
:1009F000005072696E7420535243206469736162BF
:100A00006C65640A00310A005072696E742053529A
:100A10004320656E61626C65640A00310A005061B2
:100A20007468323A20252E36732D25640A00310A67
:100A30000050617468313A20252E36732D25640AE2
:100A400000310A0044657374696E6174696F6E3AAF
:100A500020252E36732D25640A00310A0043616C6F
:100A60006C7369676E3A20252E36732D25640A0053
:100A7000310A0050617468323A20252E36732D25D4
:100A8000640A00310A0050617468313A20252E361C
:100A9000732D25640A00310A0044657374696E6120
:100AA00074696F6E3A20252E36732D25640A003145
:100AB0000A0043616C6C7369676E3A20252E3673A9
:100AC0002D25640A00310A004D6573736167652046
:100AD00073656E740A00310A004C6F636174696F4C
:100AE0006E207570646174652073656E740A0031E0
:100AF0000A005061636B65742073656E740A00317F
:100B00000A00436F6E66696775726174696F6E2063
:100B100073617665640A00300A004572726F723A3A
:100B2000204E6F2073746F72656420636F6E666908
:100B30006775726174696F6E20746F206C6F616489
:100B4000210A00436F6E66696775726174696F6E22
:100B5000206C6F616465640A00310A00436F6E6641
:100B6000696775726174696F6E20636C6561726527
:100B7000642E205265737461727420746F206C6FE0
:100B800061642064656661756C74732E0A002D2D96
:100B90002D2D2D2D2D2D2D2D2D2D2D2D2D0A004DB5
:100BA0006F64656D2072656164790A0044656661F1
:100BB000756C7420636F6E66696775726174696FB6
:100BC0006E206C6F61646564210A00756E736967DD
:100BD0006E65642E696F2F6D6963726F61707273D9
:100BE0000A004D6963726F415052532076302E32A5
:100BF000610A002D2D2D2D2D2D2D2D2D2D2D2D2D41
:100C00002D2D0A006275665F706F696E74657220C3
:100C10003E3D2062756600626572746F732F6D775A
:100C20006172652F666F726D617477722E6300203A
:100C30003D20307825700A00496E76616C69642029
:100C40007074723A20003A200041737365727469BF
:100C50006F6E206661696C65643A200011241FBEC6
:100C6000CFEFD8E0DEBFCDBF12E0A0E0B1E0E2E61A
:100C7000F1E702C005900D92A232B107D9F716E054
:100C8000A2E2B2E001C01D92AD3CB107E1F70E94C3
:100C900004170C94AF380C9400001092C00088E93F
:100CA0008093C10008951092C1000895FC0122852F
:100CB000211105C021E0228788EB8093C1000895AF
:100CC0009A01AB01CA01B901969587957795679509
:100CD000605C7D4B804F9F4F0E94A23621503109AE
:100CE0003093C5002093C4000895E2ECF0E08081C9
:100CF000A4E0660F771FAA95E1F78F7C862B80838F
:100D000008959FB7F89484B1886284B99FBF8FB764
:100D1000F894229A8FBF8FB7F89424988FBF80EDF4
:100D20008CBD8CB581608CBD8DB58E7F8DBD0895D9
:100D30001CBC9FB7F89484B1837C84B99FBF08958D
:100D400008950895FC01828508956FB7F894DC0139
:100D50001A962C911A97211120C0E0912A06F09141
:100D60002B06478D50A121A132A142175307A9F0AC
:100D700021E01A962C93A78DB0A185A196A1A81762
:100D8000B90719F483A194A104C0A78DB0A1CD0126
:100D9000019690A3878F8C918EBD6FBF0895CF93DE
:100DA000DF93EC018230910544F049E953E067E7B5
:100DB00070E088E690E00E9417342BE02C9FC00181
:100DC0002D9F900D11248A5F9E4FDF91CF91089542
:100DD0001F920F920FB60F9211242F933F938F9370
:100DE0009F93AF93BF93EF93FF93E0912806F09109
:100DF0002906278D30A181A192A12817390731F446
:100E000088E98093C1001092100113C0A78DB0A192
:100E100085A196A1A817B90719F483A194A104C0CC
:100E2000A78DB0A1CD01019690A3878F8C9180935F
:100E3000C600FF91EF91BF91AF919F918F913F912C
:100E40002F910F900FBE0F901F9018951F920F9229
:100E50000FB60F9211242F933F934F935F938F936D
:100E60009F93AF93BF93EF93FF93E0912806F09188
:100E7000290697A58091C0008871892B87A750917A
:100E8000C60027A130A583A594A52817390739F4F2
:100E900021A532A585A596A52817390761F021A5BA
:100EA00032A587A190A5019741E02817390709F0DD
:100EB00040E0842F01C081E080FF04C087A58160ED
:100EC00087A712C0A1A5B2A55C9321A532A585A5CF
:100ED00096A52817390719F483A594A503C081A501
:100EE00092A5019692A781A7FF91EF91BF91AF9133
:100EF0009F918F915F914F913F912F910F900FBED6
:100F00000F901F9018951F920F920FB60F921124F9
:100F10002F933F934F938F939F93AF93BF93EF93F1
:100F2000FF93E0912A06F0912B0627A130A583A517
:100F300094A52817390739F421A532A585A596A5CA
:100F40002817390761F021A532A587A190A501973F
:100F500041E02817390709F040E0842F01C081E003
:100F600080FD13C08EB5A1A5B2A58C9321A532A595
:100F700085A596A52817390719F483A594A503C05C
:100F800081A592A5019692A781A7E0912A06F091EA
:100F90002B06278D30A181A192A12817390799F03E
:100FA000A78DB0A185A196A1A817B90719F483A1AF
:100FB00094A104C0A78DB0A1CD01019690A3878F05
:100FC0008C918EBD02C010921B01FF91EF91BF91D9
:100FD000AF919F918F914F913F912F910F900FBEA5
:100FE0000F901F9018959FB7F89483E085BB14BCB1
:100FF00015BC82E084BD85B5836085BD16BC89EFD4
:1010000087BDEEE6F0E080818E7F80838081826004
:1010100080839FBF0895CF93DF93EC01FB015FB7FF
:10102000F894278D30A183A194A128173907E9F4FA
:1010300021A132A185A196A128173907B1F481E039
:101040005FBF80FD11C04FB7F894A1A1B2A1CC93AE
:1010500021A132A185A196A12817390799F483A16E
:1010600094A192A381A314C0DACF81A192A1278D6C
:1010700030A12150310941E08217930709F040E087
:10108000842FDECF21A132A12F5F3F4F32A321A3B6
:101090004FBF80A991A9DC01ED91FC910084F185FD
:1010A000E02D0995CE019927DF91CF910895FC019C
:1010B0004FB7F89427A130A581A592A54FBF281757
:1010C000390739F087A5897B79F024C087A5897B0A
:1010D000C9F74FB7F89427A130A581A592A54FBFB6
:1010E0002817390799F3EECF2FB7F894A7A1B0A529
:1010F00085A596A5A817B90719F483A594A504C0DA
:10110000A7A1B0A5CD01019690A787A38C912FBF71
:1011100090E008958FEF9FEF0895AF92BF92CF9226
:10112000DF92EF92FF920F931F93CF93DF937C0197
:101130005B016A01FC0100891189228933890C3421
:1011400012452544334541F04CEB50E06CE771E02B
:1011500084E691E00E941734E50100E010E00C15F0
:101160001D0559F0C7010E9457088F3F2FEF9207C6
:1011700021F00F5F1F4F8993F2CFC801DF91CF910C
:101180001F910F91FF90EF90DF90CF90BF90AF90A5
:101190000895AF92BF92CF92DF92EF92FF920F939A
:1011A0001F93CF93DF937C015B016A01FC010089EF
:1011B0001189228933890C3412452544334541F085
:1011C0004CEB50E06CE771E084E691E00E9417344C
:1011D000E50100E010E00C151D0561F08991B701F3
:1011E000992787FD90950E940B08019619F00F5FD3
:1011F0001F4FF1CFC801DF91CF911F910F91FF9049
:10120000EF90DF90CF90BF90AF900895CF93DF9392
:10121000EC01488959896A897B894C345245654477
:10122000734541F04CEB50E06CE771E084E691E0EF
:101230000E9417348FA590E0DF91CF910895CF934E
:10124000DF93EC01488959896A897B894C3452457E
:101250006544734541F04CEB50E06CE771E084E687
:1012600091E00E9417341FA6DF91CF910895CF938C
:10127000DF93EC01488959896A897B894C3452454E
:101280006544734549F04CEB50E06CE771E084E64F
:1012900091E00E94173400C02F8D38A189A19AA136
:1012A00028173907C9F788A999A9DC01ED91FC91A4
:1012B0000284F385E02D09958111EECF80E090E066
:1012C000DF91CF910895FC014FB7F89427A130A585
:1012D00081A592A54FBF28173907B1F02FB7F89411
:1012E000A7A1B0A585A596A5A817B90719F483A548
:1012F00094A504C0A7A1B0A5CD01019690A787A38E
:101300008C912FBF90E008958FEF9FEF08956FB7F6
:10131000F894FC0147A150A521A532A56FBF81E03B
:101320004217530709F480E00895DC01D0968D91AF
:101330009C91D197DC01ED91FC910480F581E02D29
:101340000994EF92FF920F931F93CF93DF93EC01D9
:101350008B016230710540F042E651E064E371E0D8
:1013600088E191E00E941734F801EE0FFF1FE85D5D
:10137000F94FD183C0838E8D882341F045E651E03B
:1013800067E071E08AEF90E00E94173481E08E8F71
:101390001D8F0C8FC8010E94CF0699AB88ABDC0172
:1013A00012968D919C911397892B41F44DE651E053
:1013B00069EE70E088ED90E00E941734E8A9F9A981
:1013C00084819581892B41F44EE651E067EC70E011
:1013D00086EB90E00E941734E8A9F9A9E680F7802F
:1013E00002811381B2E0EB16F10440F441E251E0D6
:1013F0006EE970E085E990E00E9417341CA30BA30E
:101400001AA309A318A30F8FC7010197800F911F7B
:101410009EA38DA3E8A9F9A9E084F1840481158134
:10142000E2E0EE16F10440F441E251E06EE970E0D2
:1014300085E990E00E9417341CA70BA71AA709A7FB
:1014400018A70FA3C7010197800F911F9EA78DA713
:1014500088A999A9DC01ED91FC910190F081E02D22
:10146000BE01099540E855E260E070E0CE010E94BF
:1014700095091FA6CE01DF91CF911F910F91FF908B
:10148000EF9008954FB7F894FC0121A532A530A73D
:1014900027A34FBF08954FB7F894FC0121A132A1B3
:1014A00030A3278F4FBF0895CF93DF93EC010E94A5
:1014B000420ACE01DF91CF910C944B0ACF93DF9378
:1014C000EC01488959896A897B894C3452456544C5
:1014D000734541F04CEB50E06CE771E084E691E03D
:1014E0000E9417348E8D811108C04BE851E063E5EE
:1014F00071E085E491E00E9417341E8ECE010E94B7
:10150000370988A999A9DC01ED91FC910280F3814A
:10151000E02D099519AA18AACE010E94540A80E06C
:1015200090E0DF91CF910895CF93DF93EC0148894C
:1015300059896A897B894C3452456544734541F029
:101540004CEB50E06CE771E084E691E00E941734C8
:10155000CE010E945E0A6C8D7D8DCE010E94A10994
:10156000CE01DF91CF910895FC01CB0122E3DF0191
:101570001D922A95E9F74CE452E565E473E5408B4A
:10158000518B628B738B24E93AE0358324832EE5FB
:101590003AE0378326832DE838E03183208329EC35
:1015A00038E03383228327E339E03387228726E03C
:1015B00039E0358724872FE139E037872687BC015A
:1015C000CF010C94A1091F920F920FB60F92112414
:1015D0000F931F932F933F934F935F936F937F933B
:1015E0008F939F93AF93BF93CF93DF93EF93FF932B
:1015F00080912C0690912D06A0912E06B0912F0679
:101600000196A11DB11D80932C0690932D06A093E9
:101610002E06B0932F060BEA1AEBC0916202D0910E
:10162000630288819981892BD1F18FB7F894409119
:101630002C0650912D0660912E0670912F068FBFBB
:1016400088859985AA85BB85481B590B6A0B7B0B3E
:1016500077FD25C0CF3FD10509F048F42BEC30E0F1
:1016600040EC51E063EB71E0CE010E942D34EA8141
:10167000FB818881998191838083E881F9818A81C6
:101680009B81938382831B821A82198218821B8B0F
:101690000A8BEC85FD85CE010C960995BECFFF9196
:1016A000EF91DF91CF91BF91AF919F918F917F91FA
:1016B0006F915F914F913F912F911F910F910F90DB
:1016C0000FBE0F901F90189586E692E090936302EC
:1016D0008093620210926502109264021092670277
:1016E0001092660282E692E090936902809368020B
:1016F00010922C0610922D0610922E0610922F0694
:101700000E94F30780913006882341F041E951E0BF
:1017100060EA71E08DE891E00E94173481E08093E7
:1017200030060895EF92FF920F931F93CF93DF93AC
:101730001F92CDB7DEB77C018B018983DB01129646
:101740008D919C911397892B41F44EE051E068EF05
:1017500071E08EEE91E00E941734D8011296ED915F
:10176000FC91139741E050E0BE016F5F7F4FC801CD
:101770000995019719F4C701992702C08FEF9FEFD0
:101780000F90DF91CF911F910F91FF90EF900895EF
:101790000F931F93CF93DF931F92CDB7DEB78C01CA
:1017A000DC018D919C91892B41F442EF50E06CED6E
:1017B00071E083ED91E00E941734D801ED91FC9126
:1017C00041E050E0BE016F5F7F4FC801099501976E
:1017D00019F4898190E002C08FEF9FEF0F90DF91A5
:1017E000CF911F910F910895CF93DF93CDB7DEB7BF
:1017F0009E01275F3F4F4D815E8162E97BE08F81D3
:1018000098850E94210CDF91CF9108950F931F932B
:10181000CF93DF938C01EB018991882359F0B801B4
:10182000992787FD90950E94920B8F3F2FEF92078B
:1018300099F702C080E090E0DF91CF911F910F9166
:1018400008952F923F924F925F926F927F928F9264
:101850009F92AF92BF92CF92DF92EF92FF920F933F
:101860001F93CF93DF93CDB7DEB7C45AD1090FB61C
:10187000F894DEBF0FBECDBFFC01C856DF4F7983A1
:101880006883C859D040C656DF4F59834883CA5928
:10189000D0405901C257DF4F19821882CE58D0402C
:1018A0009E012F5F3F4FC957DF4F39832883C758A9
:1018B000D040AE014A575F4FC757DF4F5983488327
:1018C000C958D0409F012F5F3F4FC456DF4F398327
:1018D0002883CC59D0408081853291F1882309F446
:1018E00027C7C656DF4F68817981CA59D040C8568C
:1018F000DF4FE881F981C859D0400995C257DF4FC1
:10190000C880D980CE58D040FFEFCF1ADF0AC55724
:10191000DF4FB982A882CB58D040C257DF4FD9825F
:10192000C882CE58D040C557DF4FA880B980CB5869
:10193000D040C456DF4FE881F981CC59D040C2CFA6
:101940008181853251F4AF014E5F5F4FC456DF4F46
:1019500059834883CC59D040C4CFC456DF4FA881A7
:10196000B981CC59D040C256DF4F1882CE59D040F1
:10197000C357DF4F1882CD58D040CF56DF4F188263
:10198000C159D040CE56DF4F1882C259D040FD0118
:101990008D918B3209F45EC060F48032E9F08332BD
:1019A00009F05FC031E0C357DF4F3883CD58D040D6
:1019B000EECF8D3251F0803309F053C041E0C25672
:1019C000DF4F4883CE59D040E2CF21E0CF56DF4FE2
:1019D0002883C159D040DBCF392D3C7F932ECE5682
:1019E000DF4F4881C259D040942ACD56DF4F5881ED
:1019F000C359D04050FB92F8CF56DF4F8881C15970
:101A0000D04080FB93F8C057DF4F9881C059D04039
:101A100090FB94F8CC56DF4FE881C459D040E0FBEE
:101A200095F8C357DF4FF881CD58D040F0FB96F8BA
:101A3000CB56DF4F2881C559D04020FB97F8892D20
:101A4000837009F0A4CF81E0CE56DF4F8883C2595E
:101A5000D0409DCF51E0CE56DF4F5883C259D04081
:101A600096CFC357DF4F9881CD58D040C056DF4F37
:101A70009883C05AD0408A3229F0DF01212C312CC2
:101A80002AE013C0C5010296D5012D903C9037FE87
:101A900009C0319421943108B1E0CF56DF4FB883AB
:101AA000C159D04031965C0112C0FD018D9190ED7D
:101AB000980F9A3060F4F1012E9F10012F9F300C87
:101AC0001124F0E32F1A3108280E311CEECFCF5627
:101AD000DF4F2881C159D040222329F0C256DF4F61
:101AE0001882CE59D04080818E3221F581818A3290
:101AF00031F0DF011196612C712C2AE009C0D5016B
:101B00006D907C90329695012E5F3F4F590115C024
:101B1000FD018D9190ED980F9A3078F4A301249FE8
:101B20003001259F700C112450E3651A7108680E6E
:101B3000711CEECF66246A94762CDF018D91883675
:101B4000D9F018F48C3459F01FC08C3641F08A3724
:101B5000D9F4C057DF4F1882C059D04006C081E089
:101B6000C057DF4F8883C059D040FD01CC56DF4FAE
:101B70001882C459D04012C0FD0191E0CC56DF4F0D
:101B80009883C459D04005C0CC56DF4F1882C45941
:101B9000D040C057DF4F1882C059D040DF011196A6
:101BA000C456DF4FB983A883CC59D0408080B5E6B6
:101BB0008B1609F408C2B815ECF023E5821609F477
:101BC00053C0281564F035E4831609F4FCC147E4DA
:101BD000841609F4F0C1882009F465C42AC053E6CC
:101BE000851671F158150CF4CBC088E5881609F4F8
:101BF0008DC01FC090E7891609F471C0981564F074
:101C0000A7E68A1609F4D7C18A160CF4DBC1B9E637
:101C10008B1609F4B5C00DC0E5E78E1609F476C041
:101C2000F8E78F1609F46DC023E7821202C0D12CA9
:101C30001DC0C557DF4FB982A882CB58D0403FC4E2
:101C4000A5014E5F5F4FC557DF4F59834883CB587F
:101C5000D040D5018C918983D12C8E010E5F1F4F0E
:101C6000FE0131965F0139C4DD24D39495012E5FC6
:101C70003F4FC557DF4F39832883CB58D040D5011C
:101C8000AD90BC90A114B10421F4A0E2AA2EA1E071
:101C9000BA2E77FE04C0F0E16F2EF7E27F2E8501A9
:101CA000DD20C1F0F8018491882309F416C4C8012D
:101CB0008A199B09861597050CF00FC40F5F1F4FFB
:101CC000F1CFC8018A199B09861597050CF005C448
:101CD0000F5F1F4FD8018C918111F3CFFEC3F50127
:101CE0003296C557DF4FF983E883CB58D040D501F2
:101CF0006D917C9180E090E0ECE7EE2EE1E0FE2E2D
:101D00002BC07CE8E72E71E0F72E04C06CE7E62ECE
:101D100061E0F62EC057DF4FB881C059D040BB23D9
:101D200071F0F5013496C557DF4FF983E883CB583E
:101D3000D040D5016D917D918D919C910DC0C501D3
:101D40000296F50160817181C557DF4F99838883C1
:101D5000CB58D04080E090E021E0CD56DF4F288383
:101D6000C359D04035E7831205C0CD56DF4F1882E6
:101D7000C359D040CE56DF4F1882C259D04042C01E
:101D8000C057DF4F4881C059D040442371F0C5018E
:101D90000496C557DF4F99838883CB58D040D5012F
:101DA0006D917D918D919C910FC0F5013296C55733
:101DB000DF4FF983E883CB58D040D5016D917C91FA
:101DC000882777FD8095982F97FF13C09095809571
:101DD000709561957F4F8F4F9F4FCD56DF4F188283
:101DE000C359D040B2E0CE56DF4FB883C259D0407D
:101DF00005C0CD56DF4F1882C359D0405CE7E52EB1
:101E000051E0F52EE1E0CB56DF4FE883C559D040D5
:101E1000611571058105910529F4CB56DF4F1882B4
:101E2000C559D0406114710441F4CB56DF4FF8819D
:101E3000C559D040FF2309F47CC0CD56DF4F28811F
:101E4000C359D0408E010A571F4F2130A9F02AE014
:101E500030E040E050E00E94A236F701E60FF71FA5
:101E60008081D8018E938D01B901CA016115710578
:101E70008105910561F715C0FB01EF70FF27EE0D9D
:101E8000FF1D2081F80122938F0144E096958795EC
:101E9000779567954A95D1F761157105810591058B
:101EA00059F777FE49C0C256DF4FF881CE59D0406E
:101EB000FF2309F441C0292D2C7F922ECE56DF4FEF
:101EC0003881C259D040932ACD56DF4F4881C3593B
:101ED000D04040FB92F8CF56DF4F5881C159D040D7
:101EE00050FB93F8C057DF4F8881C059D04080FB2A
:101EF00094F8CC56DF4F9881C459D04090FB95F8A8
:101F0000C357DF4FA881CD58D040A0FB96F8CB56E1
:101F1000DF4FB881C559D040B0FB97F8292D237009
:101F200081E090E011F480E090E03101681A790AD4
:101F300003C08E010A571F4FC757DF4F8881998111
:101F4000C958D040801B910BF80120E35F01861532
:101F500097051CF422930196F9CFC357DF4FE88110
:101F6000CD58D040EE23A1F0CB56DF4FF881C559B4
:101F7000D040FF2369F0882D8F7D883549F4F50125
:101F80003197808222E0A21AB10880E3D5018C93B8
:101F9000C957DF4FE881F981C758D040AE16BF0658
:101FA00008F095C247EB52E06DE172E08AE092E002
:101FB0000E9417348CC28A948A9411E061147104CF
:101FC00049F002C0812C10E077FE07C026E0622EA7
:101FD000712C03C066246394712C95012C5F3F4FD4
:101FE000C557DF4F39832883CB58D040D501CD90DA
:101FF000DD90ED90FC9020E030E0A901C701B60132
:102000000E94B73487FF0AC0F7FAF094F7F8F0940B
:10201000B2E0CE56DF4FB883C259D040C156DF4F31
:102020001883CF59D040AA24A394B12CAC0EBD1E66
:10203000A20CB31C20E030E040E85FE3C701B6012A
:102040000E94063687FD32C0412C512C27EB33E429
:102050004AEB51E5C701B6010E94063687FD0EC066
:1020600029EF32E045E150E5C701B6010E94BB34DB
:102070006B017C01EAE04E0E511CE8CF20E030E01D
:1020800040E251E4C701B6010E94063687FD49C00F
:1020900020E030E040E251E4C701B6010E94BB34C9
:1020A0006B017C01FFEF4F1A5F0AE8CF20E030E0C0
:1020B000A901C701B6010E94B734412C512C8823D5
:1020C00081F12FEF36EE4BED5EE2C701B6010E94C3
:1020D000B734181674F029EF32E045E150E5C70136
:1020E000B6010E940A366B017C012AE0421A5108AF
:1020F000E8CF20E030E040E85FE3C701B6010E948E
:10210000B73487FF0EC020E030E040E251E4C70161
:10211000B6010E940A366B017C0131E0431A510876
:10212000E8CF112301F14614570444F44CEF441650
:102130004FEF54061CF064187508812C51E0651AA5
:10214000710881E0C357DF4F9881CD58D040982760
:10215000C156DF4F9883CF59D040A1E0C357DF4F1E
:10216000A883CD58D04081104BC057FE3DC080E3BE
:10217000E1E0F0E0EC0FFD1FE20DF31D8083F501BF
:102180006114710459F4C357DF4FB881CD58D04062
:10219000B11104C0319680E090E006C032968EE224
:1021A000D50111968C93C30192012F5F3F4F280FE9
:1021B000391F40E38F018217930729F0009719F028
:1021C00041930197F7CF930120953095421653061E
:1021D0000CF4D1C03C01E1E0F0E0CA56DF4FF983D6
:1021E000E883C659D0405CC022273327241935091B
:1021F000CA56DF4F39832883C659D040850150C065
:102200008501CA56DF4F19821882C659D04048C08E
:10221000C701B6010E942335CF55DF4F688379830C
:102220008A839B83C15AD040CF55DF4F4881598163
:10223000C15AD040BA01882777FD8095982F0E9417
:1022400056359B01AC01C701B6010E94523420E013
:1022500030E040E251E40E940A366B017C019801B3
:102260002F5F3F4FCF55DF4F8881C15AD040805DEF
:10227000D8018C93CA56DF4F88819981C659D040C6
:102280000196CA56DF4FE881F981C659D040EF2B3D
:1022900091F0CA56DF4F99838883C659D04089018F
:1022A000CA56DF4F28813981C659D040621673065D
:1022B0000CF0AECF14C06114710439F4C357DF4F72
:1022C000F881CD58D040FF2339F098012E5F3F4F61
:1022D000EEE2D8011196EC9381E090E0DACF20E0B5
:1022E00030E040EA50E4C701B6010E94063687FD9F
:1022F00042C0F80181E090E030E322912E3251F0AB
:10230000820F8A3321F0808380E090E003C0308325
:1023100081E090E0AE16BF0680F3892B61F1882042
:10232000B9F0F801AE16BF0678F4DF018E919D0179
:102330008E3239F4CF010297DC018C918083F90150
:1023400001C080833197EECFBFEF4B1A5B0A0BC001
:102350000F5F1F4FF801AE16BF0628F4DF018E9104
:102360008083FD01F8CF81E3E1E0F0E0EC0FFD1F99
:10237000E20DF31D8083C156DF4FE881CF59D04075
:10238000EE2349F0F8018291803311F48F01FACFE6
:102390008E3209F48F018820B1F1D8018C92C801E6
:1023A000029657FE07C02DE211962C93519441944A
:1023B000510803C02BE2F80121838C01065F1F4FF7
:1023C00020E030E02F5F3F4FF8013196C2016AE014
:1023D00070E00E948E36805DD8018C932B016115D0
:1023E000710511F08F01EECF22303105DCF3E21BD5
:1023F000F30B199781918E93215031091216130610
:10240000CCF309501109C256DF4FB881CE59D040E4
:10241000BB2309F461C0E92DEC7F9E2ECE56DF4F21
:10242000F881C259D0409F2ACD56DF4F2881C35929
:10243000D04020FB92F8CF56DF4F3881C159D040B1
:1024400030FB93F8C057DF4F4881C059D04040FB64
:1024500094F8CC56DF4F5881C459D04050FB95F8C2
:10246000C056DF4F8881C05AD04080FB96F8CB56CB
:10247000DF4F9881C559D04090FB97F8292D2370E4
:1024800081E090E011F480E090E09101281B390B8D
:10249000F50140E35F01C8018E1B9F0B8217930774
:1024A000DCF44293F7CFC557DF4FB982A882CB58EF
:1024B000D040C456DF4FF983E883CC59D040D12CAB
:1024C0000FE111E08CE1A82E81E0B82E06C0D12CDE
:1024D0008E010A571F4F01C0D12C0A191B09201663
:1024E00031060CF440C0A92DAC7F9A2ECE56DF4F9A
:1024F000B881C259D0409B2ACD56DF4FE881C359DD
:10250000D040E0FB92F8CF56DF4FF881C159D04060
:10251000F0FB93F8C057DF4F2881C059D04020FB13
:1025200094F8CC56DF4F3881C459D04030FB95F831
:10253000C056DF4F4881C05AD04040FB96F8CB567A
:10254000DF4F5881C559D04050FB97F87101E01A10
:10255000F10A292D237081E090E011F480E090E0F1
:10256000E81AF90A02C0E12CF12CCF56DF4F88811E
:10257000C159D040811122C031E0E31AF108F7FCC3
:102580001DC0C656DF4F68817981CA59D04080E2AC
:10259000C856DF4FE881F981C859D0400995C25724
:1025A000DF4F28813981CE58D0402F5F3F4FC2572F
:1025B000DF4F39832883CE58D040DECF492D4C7F62
:1025C000942ECE56DF4F5881C259D040952ACD5611
:1025D000DF4F8881C359D04080FB92F8CF56DF4F40
:1025E0009881C159D04090FB93F8C057DF4FA88124
:1025F000C059D040A0FB94F8CC56DF4FB881C459E5
:10260000D040B0FB95F8C056DF4FE881C05AD040AB
:10261000E0FB96F8CB56DF4FF881C559D040F0FB70
:1026200097F8892D837001F1813011F48BE201C09C
:102630008DE2C656DF4F68817981CA59D040C856AD
:10264000DF4FE881F981C859D0400995C257DF4F63
:1026500028813981CE58D0402F5F3F4FC257DF4F7E
:1026600039832883CE58D040D1100AC03501C257D3
:10267000DF4FA880B980CE58D040A618B70821C037
:10268000C257DF4FC880D980CE58D040AC18BD08A3
:102690000150110917FD2DC0F501EC0DFD1D8491B0
:1026A000C656DF4F68817981CA59D040C856DF4F7E
:1026B000E881F981C859D0400995FFEFCF1ADF0AA8
:1026C000E7CF6501C60CD71C0150110917FD11C0D9
:1026D000C656DF4F68817981CA59D040D3018D91A8
:1026E0003D01C856DF4FE881F981C859D0400995AE
:1026F000E8CFCF56DF4FF881C159D040FF2309F40E
:102700000CC921E0E21AF108F7FC07C9C656DF4FF1
:1027100068817981CA59D04080E2C856DF4FE8818C
:10272000F981C859D0400995FFEFCF1ADF0AE9CFE8
:10273000C257DF4F88819981CE58D040CC55DF4FAA
:102740000FB6F894DEBF0FBECDBFDF91CF911F91C2
:102750000F91FF90EF90DF90CF90BF90AF909F9040
:102760008F907F906F905F904F903F902F90089543
:10277000CF92DF92EF92FF920F931F93CF93DF934D
:102780001F92CDB7DEB77C01462F82E8860F9701F6
:10279000265B3E4F6901823010F06B3149F4F6013F
:1027A000608171818BE190E049830E94920B4981A5
:1027B000D701A05BBE4F2C9111965C911197842F8D
:1027C00090E0FC01E227EE0FFF1FED5CFC4F25912E
:1027D0003491052F10E0202731272D933C93F601EB
:1027E000608171810F90DF91CF911F910F91FF90C8
:1027F000EF90DF90CF900C94920B2F923F924F92DC
:102800005F926F927F928F929F92AF92BF92CF9280
:10281000DF92EF92FF920F931F93CF93DF93CDB789
:10282000DEB7C455D1090FB6F894DEBF0FBECDBFD9
:102830008C014C0126EB821A2EEF920A5C014BEAC6
:10284000A41A4EEFB40A7C0184EBE81A8EEFF80A62
:10285000D4018D919C910E94C80B8F3FBFEF9B07C5
:1028600009F425C1F50120812111F0C08E379105B1
:1028700009F0DEC0D7014D915C91F801E25BFE4F9B
:102880001F014231510508F4C5C080819181883B08
:10289000904F09F0BFC0D801FE013896CE010E96C8
:1028A0002D912695203209F420E02193E817F907AD
:1028B000B9F7D80116968C91169786958F708E87EA
:1028C0001796FE013196CF0106962D91269520325E
:1028D00009F420E02193E817F907B9F7F8013D96CC
:1028E000D8011D968C9186958F708F8329964FAC59
:1028F0002997512C61E070E0808180FF10C02896FC
:102900005FAE289729964FAE2997818190E02B964C
:102910009FAF8EAF2B97039709F07CC05AC0B7E0EA
:10292000B51568F366246394712C6C0E7D1E27E048
:10293000529E600C711C1124CF01019663969FAFCB
:102940008EAF639780E090E0252D30E06396AEADCA
:10295000BFAD6397DD906396BFAFAEAF6397D6947C
:10296000B0E2DB1202C0C12C01C0CD2CD301A80FF4
:10297000B91F1E96CC9201968630910539F737968D
:102980009081B7E0CB2EC29ED001C39EB00D112422
:10299000CC24C394D12CCC0EDD1EAC0DBD1D892FD3
:1029A00086958F7054968C9397FF08C0CB0102C018
:1029B000880F991F2A95E2F7482A09C0DB0102C057
:1029C000AA0FBB1F2A95E2F79D012095422253943E
:1029D00093CF82812C968FAF2C97803FD9F433967A
:1029E00042505109C8018E1B9F0B480F591F60961A
:1029F0005FAF4EAF60972E96FFAFEEAF2E97F80108
:102A0000EE5AFE4F0190F081E02D309719F0CE0183
:102A10000196099581E0F801EC5AFE4F80838FEF13
:102A20009FEFD1018D939C93F7011182108210CFFB
:102A30008F37910529F4F801EC5AFE4F108208CF28
:102A40008B31910519F481E0808302CFF801EC5AB3
:102A5000FE4F2081222341F1D7012D913C912A3450
:102A6000B1E03B0700F5A9014F5F5F4FF7015183CC
:102A70004083F801E20FF31F8083D801A25BBE4FB1
:102A80002D913C911197F901E827FF27EE0FFF1FC9
:102A9000ED5CFC4F85919491232F33278227932758
:102AA0008D939C9301C01082D5011C92D1CEF4016C
:102AB00000811181D8011C968D919C911D97892BC5
:102AC00041F449E451E061E273E087E193E00E9460
:102AD0001734D8011C96ED91FC911D97C8010995FA
:102AE000892BC9F0F40100811181D8011E968D91C6
:102AF0009C911F97892B41F442E551E065E073E01A
:102B000088EF92E00E941734D8011E96ED91FC9157
:102B10001F97C8010995CC5ADF4F0FB6F894DEBF56
:102B20000FBECDBFDF91CF911F910F91FF90EF901E
:102B3000DF90CF90BF90AF909F908F907F906F90DD
:102B40005F904F903F902F9008952F923F924F9219
:102B50005F926F927F928F929F92AF92BF92CF922D
:102B6000DF92EF92FF920F931F93CF93DF93CDB736
:102B7000DEB72C970FB6F894DEBF0FBECDBF9C8793
:102B80008B877B015A01288739871D830C83611548
:102B9000710541F44BEE50E066EE72E081EE92E09A
:102BA0000E94173422E0A216B10440F44CEE50E02B
:102BB0006FEC72E081EC92E00E9417344B845C84ED
:102BC00080EB481A8EEF580A8FEF9FEFF201918346
:102BD00080836B847C84F6EB6F1AFEEF7F0AF3012F
:102BE000608171818EE790E00E94920BC12CD12C04
:102BF000C50101979F838E83CA14DB0409F468C062
:102C000021E029838E819F81C816D90609F0198297
:102C1000F70101900020E9F78F01015011090E1909
:102C20001F090730110510F006E010E0C8018E0DF5
:102C30009F1D9B838A8317018A819B8128163906F1
:102C400001F1F10121911F01822E912CC4012A87EB
:102C50000E943C382A85892B51F4203241F04EECF9
:102C600050E06CE772E085E692E00E941734C40100
:102C70000E945038682F660F8B859C850E94B81380
:102C8000DBCF0630110599F0812C912CE6E0F0E0C5
:102C9000E01BF10B8F018016910648F460E48B85F0
:102CA0009C850E94B813FFEF8F1A9F0AF4CF898189
:102CB0008066F7016681660F682B8B859C850E9474
:102CC000B813FFEFCF1ADF0A27E0E20EF11C94CF12
:102CD00063E08B859C850E94B81360EF8B859C8593
:102CE0000E94B81308851985EC80FD80E00EF11E66
:102CF0000E151F0541F0F80161918F018B859C85B0
:102D00000E94B813F5CFF2016081118160958B8527
:102D10009C850E94B813612F60958B859C850E94CD
:102D2000B813F20180819181883B904F41F045E0DA
:102D300051E06FEA72E08EE892E00E941734F301EE
:102D4000608171818EE790E02C960FB6F894DEBF1B
:102D50000FBECDBFDF91CF911F910F91FF90EF90EC
:102D6000DF90CF90BF90AF909F908F907F906F90AB
:102D70005F904F903F902F900C94920BEF92FF92A8
:102D80000F931F93CF93DF93EC018B017A01009790
:102D900041F441E251E063E572E08FE492E00E9489
:102DA00017340115110541F442E251E06DE372E080
:102DB00085E392E00E94173486E591E0FE019C01D4
:102DC000119221503040E1F7FE01E65BFE4F118386
:102DD0000083FE01EE5AFE4FF182E082FE01E05BCD
:102DE000FE4F8FEF9FEF91838083C25BDE4F99830D
:102DF0008883DF91CF911F910F91FF90EF900895FD
:102E00006AEB73E00C94E81F78940E94640B60E016
:102E100070E08AEB93E00E94B40A40E855E260E07B
:102E200070E08AEB93E00E94950986E08093C200EF
:102E300060E070E082E495E00E94B81C40E057E159
:102E400062E475E08CEE93E00E94BE168CEE93E097
:102E50000E94791E8FB7F894C0902C06D0902D0652
:102E6000E0902E06F0902F068FBFC1E08CEE93E02D
:102E70000E94FD1380916A0281112EC08AEB93E0BB
:102E80000E948709882341F18AEB93E00E9463093D
:102E900080936D0290936E0220916B0230916C02D0
:102EA000F901E159FD4FA9014F5F5F4F80835093B6
:102EB0006C0240936B022934314010F0C0936A02D7
:102EC0008FB7F894C0902C06D0902D06E0902E0677
:102ED000F0902F068FBF1BC080916B0290916C0207
:102EE000892BA9F02FB7F89480912C0690912D068C
:102EF000A0912E06B0912F062FBF8C199D09AE0907
:102F0000BF090397A105B10514F0C0936A0280912F
:102F10006A02882309F4AACF60916B0270916C0257
:102F20002CEE33E04AEB53E08FE692E00E94092456
:102F300010926A0210926C0210926B0297CFCF939C
:102F4000DF93EC0170931D0660931C06863091059B
:102F500044F041E250E06BE375E083E395E00E94CA
:102F600017341092800089E18093810081E896E017
:102F700090938700809386008C2F806480937C00E0
:102F800087B121E030E001C0220FCA95EAF7922F05
:102F90009095892387B988B1892388B980917E006B
:102FA000822B80937E0087E080937B008CEE809361
:102FB0007A00DF91CF9108951F920F920FB60F9272
:102FC00011242F933F934F935F936F937F938F932E
:102FD0009F93AF93BF93EF93FF9380E286BB609183
:102FE0007800709179007695679576956795605829
:102FF00080911C0690911D060E94CF198091320687
:10300000882349F080911C0690911D060E949F1B09
:10301000807F886007C080913106882311F088E89E
:1030200001C080E88BB9FF91EF91BF91AF919F9163
:103030008F917F916F915F914F913F912F910F9061
:103040000FBE0F901F901895AF92BF92CF92DF9254
:10305000EF92FF920F931F93CF93DF936C01EB01DD
:103060007A01DC0150960D911D912D913C91539761
:103070000D341B442345364441F04EE650E062E6F1
:1030800075E08CE495E00E9417345E01CE018E0D50
:103090009F1DF601EB57FF4FA816B90671F4C50145
:1030A0008C1B9D0BDF91CF911F910F91FF90EF90A3
:1030B000DF90CF90BF90AF9008956FB7F8944081A4
:1030C0005181228133816FBF4217530741F32FB7DC
:1030D000F894C0902C06D0902D06E0902E06F0902B
:1030E0002F062FBF6FB7F894408151812281338121
:1030F0006FBF42175307A9F44FB7F89400912C06FD
:1031000010912D0620912E0630912F064FBF0C19DD
:103110001D092E093F09101611061206130614F791
:10312000BECF6FB7F8942081318146815781241733
:10313000350719F44481558105C020813181A901E9
:103140004F5F5F4F51834083D9012C916FBFD501F1
:103150002D935D01A1CF2F923F924F925F926F927C
:103160007F928F929F92AF92BF92CF92DF92EF9217
:10317000FF920F931F93CF93DF93EC017B016A01C2
:1031800088899989AA89BB898D349B44A345B64413
:1031900041F04EE650E062E675E08CE495E00E9476
:1031A0001734870137016C0C7D1C222423946E0197
:1031B00087E7C80ED11C80E4482E512C90E4892E5C
:1031C0009FE1992EA12CB12C0615170509F477C0A3
:1031D0004FB7F8942FA538A98BA99CA928173907B0
:1031E00039F429A93AA98DA99EA92817390761F0B0
:1031F00029A93AA98FA598A9019751E0281739075D
:1032000009F050E0852F01C081E04FBF80FDE0CF85
:10321000F80181918F014FB7F894E9A9FAA9808349
:1032200029A93AA98DA99EA92817390719F48BA9AC
:103230009CA903C089A99AA901969AAB89AB4FBFF3
:10324000F6018081811121C05EA64DA61CA61BA699
:103250001AA62082299A2091550130915601409159
:10326000570150915801A0EBB4E00E94833660569C
:10327000704F8F4F9F4FA50194010E94A2363BA330
:103280002AA35B9AF1E0F09332063FB6F8942091BE
:103290005101309152014091530150915401A0EBE2
:1032A000B4E00E9483366056704F8F4F9F4FA50148
:1032B00094010E94A2363DA32CA33FBE85CFC80136
:1032C0008E199F09DF91CF911F910F91FF90EF9081
:1032D000DF90CF90BF90AF909F908F907F906F9036
:1032E0005F904F903F902F900895CF93DF93EC0124
:1032F000488959896A897B894D345B4463457644A2
:1033000041F04EE650E062E675E08CE495E00E9404
:103310001734C958DF4F88818111FDCF80E090E0DC
:10332000DF91CF910895CF93DF93EC0148895989BC
:103330006A897B894D345B446345764441F04EE6AF
:1033400050E062E675E08CE495E00E9417342FB7F8
:10335000F894C852DF4F888199812FBFDF91CF91B8
:103360000895CF93DF93EC01488959896A897B8955
:103370004D345B446345764441F04EE650E062E6EE
:1033800075E08CE495E00E9417348FB7F894C8522A
:10339000DF4F198218828FBFDF91CF910895EF928E
:1033A000FF920F931F93CF93DF93FC018C01015386
:1033B0001F4FD8014D915C91DC01A353BF4F4D933A
:1033C0005C93DC01A858BF4F8D919C911197169684
:1033D0002D913C9117978217930729F414962D91FC
:1033E0003C91159706C08D919C9111979C012F5F80
:1033F0003F4F11963C932E93EC01288126029001B9
:1034000011243595279535952795E801398328832B
:103410007F01D3EDED0EF11CE701888199818F01C9
:103420000F521F4FE8019983888395958795840FE4
:10343000951F820F931FE70199838883AF014B5239
:103440005F4F21E0181619060CF020E0EA01888190
:10345000880F822B888312968D919C911397EC0193
:10346000688312962D913C91139716968D919C919D
:1034700017972817390729F414968D919C91159761
:1034800005C012968D919C911397019613969C936B
:103490008E931297DA019C91892F869586958927BC
:1034A0008370DF01AA52BF4F833039F48C91803290
:1034B00014F48F5F01C081508C938C91885F8C9342
:1034C00080340CF435C18F738C93DF01A952BF4F48
:1034D0008C91880F97702BEF290F233010F09330C9
:1034E00009F481608C939C91892F8695892780951A
:1034F0008170968D990F892B868F8E3709F04EC07B
:10350000DF01AB57BF4F2D913C91119714968D91D0
:103510009C9115972817390759F412962D913C91D3
:10352000139716968D919C9117972817390779F064
:1035300012962D913C9113978D919C911197019723
:1035400041E02817390709F040E0842F01C081E0ED
:1035500080FDDDC01296CD91DC9113978EE78883B4
:1035600012962D913C91139716968D919C911797D9
:103570002817390729F414968D919C91159705C049
:1035800012968D919C911397019613969C938E930E
:10359000129781E081A32A9A41E0BCC0982F9F77BF
:1035A0009F3719F411A22A98C3C091A1992309F455
:1035B000BFC0982F9F739E3309F4BAC080FF03C029
:1035C00080A1806880A3878D8F5F878F90A18830CE
:1035D00008F4ACC0DF01AB57BF4F82E8890F8230DF
:1035E00018F09B3109F04BC02D913C911197149626
:1035F0008D919C9115972817390759F412962D91A2
:103600003C91139716968D919C911797281739071F
:1036100079F012962D913C9113978D919C91119771
:10362000019741E02817390709F040E0842F01C0D5
:1036300081E080FD20C01296CD91DC9113978BE143
:10364000888312962D913C91139716968D919C919B
:1036500017972817390729F414968D919C9115977F
:1036600005C012968D919C911397019613969C9389
:103670008E93129704C011A22A9840E001C041E045
:103680002D913C91119714968D919C911597281727
:10369000390759F412962D913C91139716968D91F6
:1036A0009C9117972817390779F012962D913C9124
:1036B00013978D919C911197019751E02817390725
:1036C00009F050E0852F01C081E080FD20C080A17D
:1036D0001296CD91DC911397888312962D913C918F
:1036E000139716968D919C9117972817390729F4EF
:1036F00014968D919C91159705C012968D919C9171
:103700001397019613969C938E93129703C011A260
:103710002A9840E010A2178E41110AC0E852FF4FCC
:103720008081918181609183808302C0969590A36E
:10373000DF91CF911F910F91FF90EF900895DC01E1
:1037400096968C9196978111EAC098968C9198974D
:103750008111A0C09F962D913C91D097D1968D91CB
:103760009C91D2972817390739F494968D919C91A2
:103770009597892B09F45CC099968C919997811142
:1037800003C09A961C929A9781E099968C93999788
:1037900092968D919C919397009789F59F962D9184
:1037A0003C91D097D1968D919C91D297281739074B
:1037B00051F494968D919C919597019795969C9331
:1037C0008E93949721C09F96ED91FC91D097D596BA
:1037D0008D919C91D697E817F90729F4D3968D918E
:1037E0009C91D49706C09F96ED91FC91D097CF0104
:1037F0000196D0969C938E939F97808106C00197E7
:1038000093969C938E9392978EE797968C93979727
:1038100097968C9197978B3199F59F962D913C9126
:10382000D097D1968D919C91D2972817390749F45A
:103830005B9810923206A958BF4F1C92299880E0DD
:1038400008959F96ED91FC91D097D5968D919C917E
:10385000D697E817F90729F4D3968D919C91D497C0
:1038600006C09F96ED91FC91D097CF010196D0961E
:103870009C938E939F97808197968C93979706C081
:103880008E57823018F499961C92999781E09896F9
:103890008C93989799962C9199979D968D919C9140
:1038A0009E972223A9F09A962C919A97253080F022
:1038B0009A961C929A978034910519F485E790E0C6
:1038C00002C080E490E09E969C938E939D9723C0C7
:1038D00098963C91989797962C919797232341F02F
:1038E0009A968C919A978F5F9A968C939A970FC01D
:1038F0009A961C929A978034910519F485E790E086
:1039000002C080E490E09E969C938E939D97330F27
:1039100098963C93989788E096968C9396979D9668
:10392000ED91FC919E979B968D919C919C97E80FB1
:10393000F91F9F0131709C963C932E939B9796960E
:103940008C919697815096968C93FF27E038F105DD
:1039500030F08FEF90E0AC014E1B5F0BFA01E159A4
:10396000FA4F84912F3F310511F008F080950895AA
:10397000CF93DF93EC01CB012AEDFE0111922A9542
:10398000E9F77D8F6C8F20E430E03EA72DA79E01E4
:1039900020583F4FFE01E858FF4F3583248333837F
:1039A0002283318320839E012C573F4F3783268308
:1039B0009E0123573F4FDE01AB57BF4F15963C93F7
:1039C0002E93149713963C932E93129711963C9333
:1039D0002E939E0124533F4F17963C932E93169798
:1039E0009E01295C3F4F3CAB2BAB3AAB29AB38ABCC
:1039F0002FA79E012A583F4F3EAB2DAB24E030E06D
:103A0000A281B3811C9262817381468157816417C0
:103A1000750719F44481558104C0428153814F5F79
:103A20005F4F53834283215031092115310541F7FE
:103A3000BE010E949F178AB1886F8AB9219A229A83
:103A40004DE45BE463E576E4488B598B6A8B7B8BB2
:103A50008BEA98E19B838A8384E298E19983888347
:103A600085E799E19B878A8783E999E19D878C8720
:103A700081EB99E19F878E87DF91CF9108956FEF5A
:103A80008EE290E00E94973880914B01882341F0AC
:103A90008CE59BE09F938F930E9495330F900F903E
:103AA00080914B0181110CC080912706811108C0C3
:103AB00089E59BE09F938F930E9495330F900F9021
:103AC0000895CF938EE290E00E947938893609F00C
:103AD000E3C046E050E068E270E085E491E00E94D7
:103AE000693846E050E062E270E08FE391E00E94C6
:103AF000693846E050E06CE170E089E391E00E94B3
:103B0000693846E050E066E170E081E391E00E94B0
:103B1000693885E190E00E94793890E0909324061E
:103B20008093230684E190E00E94793890E090939E
:103B300022068093210683E190E00E94793890E08C
:103B4000909338018093370182E190E00E947938A8
:103B500090E09093300180932F0181E190E00E94EA
:103B6000793891E0811101C090E09093500180E19B
:103B700090E00E94793891E0811101C090E090932B
:103B80004F018FE090E00E94793891E0811101C0EF
:103B900090E090934E018EE090E00E94793891E0A1
:103BA000811101C090E090934D018DE090E00E9462
:103BB000793891E0811101C090E090934C018CE044
:103BC00090E00E947938C1E0811101C0C0E0C0934B
:103BD0004B018BE090E00E94793891E0811101C0A7
:103BE00090E0909327068AE090E00E9479388093D5
:103BF0002C0189E090E00E94793880932B0188E0C5
:103C000090E00E94793880932A0187E090E00E943A
:103C100079388093290186E090E00E94793880937A
:103C20002E0185E090E00E94793880932D0184E098
:103C300090E00E94793891E0811101C090E090936A
:103C40001E0682E090E00E948138A0E0B0E0809300
:103C5000550190935601A0935701B093580180E00D
:103C600090E00E948138A0E0B0E0809351019093F1
:103C70005201A0935301B0935401CC23C1F1809120
:103C800026068823A1F183E49BE09F938F930E94F3
:103C900095330F900F902BC080912606882381F0DA
:103CA0008091270681110CC080914B01882341F03F
:103CB0008AE19BE09F938F930E9495330F900F9022
:103CC00080912606882381F08091270681110CC0FF
:103CD00080914B01811108C087E19BE09F938F93F6
:103CE0000E9495330F900F9081E080932506CF912D
:103CF000089590936606809365060E94611D81E099
:103D00008093260680914B018823E9F12FEF85EA05
:103D10009EE0215080409040E1F700C0000083EF1A
:103D20009BE09F938F930E94953382EE9BE09F933D
:103D30008F930E9495338BEC9BE09F938F930E940F
:103D400095330F900F900F900F900F900F908091E0
:103D50002506882341F08CEA9BE09F938F930E9475
:103D600095330F900F908FE99BE09F938F930E9464
:103D700095338EE89BE09F938F930E9495330F902D
:103D80000F900F900F90089546E050E068E270E0C9
:103D900085E491E00E94873846E050E062E270E0FE
:103DA0008FE391E00E94873846E050E06CE170E0DC
:103DB00089E391E00E94873846E050E066E170E0D8
:103DC00081E391E00E9487386091230685E190E0CD
:103DD0000E9497386091210684E190E00E94973814
:103DE0006091370183E190E00E94973860912F0144
:103DF00082E190E00E9497386091500181E190E06B
:103E00000E94973860914F0180E190E00E949738BE
:103E100060914E018FE090E00E94973860914D01D3
:103E20008EE090E00E94973860914C018DE090E028
:103E30000E94973860914B018CE090E00E94973887
:103E4000609127068BE090E00E94973860912C01EA
:103E50008AE090E00E94973860912B0189E090E021
:103E60000E94973860912A0188E090E00E9497387C
:103E70006091290187E090E00E94973860912E01BF
:103E800086E090E00E94973860912D0185E090E0F7
:103E90000E94973860911E0684E090E00E94973857
:103EA000609155017091560182E090E00E94A9381E
:103EB000609151017091520180E090E00E94A93818
:103EC00069E68EE290E00E94973880914B0188234A
:103ED00041F082E09BE09F938F930E9495330F9077
:103EE0000F9080914B0181110CC0809127068111A8
:103EF00008C08FEF9AE09F938F930E9495330F90A5
:103F00000F9008950F931F939C01CA0146E0EFE3C1
:103F1000F1E0A1E5B6E001900D924A95E1F74091FC
:103F200021064093570646E0E5E4F1E0A2EBB6E057
:103F300001900D924A95E1F7409123064093B8060F
:103F400046E0E9E3F1E0A8E5B6E001900D924A957C
:103F5000E1F74091370140935E0646E0E1E3F1E08E
:103F6000A2ECB6E001900D924A95E1F740912F0145
:103F70004093C80647E0E1E5F6E0A3E3B6E0019030
:103F80000D924A95E1F747E0E2EBF6E0AAE3B6E0EE
:103F900001900D924A95E1F747E0E8E5F6E0A1E4EB
:103FA000B6E001900D924A95E1F747E0E2ECF6E0C9
:103FB000A8E4B6E001900D924A95E1F78B0144E048
:103FC00050E063E376E00E94A5151F910F910895DC
:103FD0006F927F928F929F92AF92BF92CF92DF9219
:103FE000EF92FF920F931F93CF93DF9300D000D0F7
:103FF00000D0CDB7DEB78C013B0180915001882302
:10400000E9F080914C01882329F06CE971E0C3014B
:104010000E94060CD80116968C911F928F931F93C5
:104020000F9382EA91E09F938F937F926F920E9409
:10403000F40B0FB6F894DEBF0FBECDBF80914F01D9
:10404000882331F180914C01882361F08DEA91E061
:104050009F938F937F926F920E94F40B0F900F901B
:104060000F900F90D8011D968C911F928F93C801CD
:1040700007969F938F9382EA91E09F938F937F920D
:104080006F920E94F40B0FB6F894DEBF0FBECDBF47
:1040900080914E01811105C080914D01811137C081
:1040A0005AC080914C01882329F063EB71E0C30171
:1040B0000E94060C7801FEE0EF0EF11CC12CD12C01
:1040C000480126E4820E911C82EAA82E81E0B82ED7
:1040D000D4018C9190E0C816D906F4F6D701169653
:1040E0008C911F928F93FF92EF92BF92AF927F922B
:1040F0006F920E94F40BBFEFCB1ADB0AE7E0EE0EE3
:10410000F11C0FB6F894DEBF0FBECDBFE1CF80919A
:104110004C01882329F06AEB71E0C3010E94060C70
:10412000F801E55BFF4F81818F9380818F93F801C8
:10413000E35BFF4F81818F9380818F9321EC31E08E
:104140003F932F937F926F920E94F40B0FB6F894D7
:10415000DEBF0FBECDBF66EC71E0C3010E94060C4E
:1041600080911E06882309F4EBC0F801E35BFF4F42
:104170000190F081E02DEC30F10508F4E1C0D801A8
:10418000A55BBF4F2D913C915F01A20EB31E80E055
:1041900090E0C12CD12CAE014F5F5F4FD5016E91E5
:1041A0005D016B3769F4DA01B501FB01F190BF01E4
:1041B000FD927D01E41AF50A8E159F05B0F76C019A
:1041C00001968730910551F7C114D10409F4B8C0A4
:1041D00081E090E0A1E0F901E80FF91F608170E053
:1041E000FC01EC5BFE4F4081552747FD509564175D
:1041F000750719F087E090E0A0E0019687309105FF
:1042000054F340E050E0F901E80FF91F60816D328E
:1042100009F4AC0101968A309105ACF341155105C2
:10422000A1F0F901E40FF51F8281609123067091DE
:104230002406803221F4818190E0C09702C090E092
:1042400086978617970709F07BC0AA2309F478C0E0
:104250005601FEE0AF0EB11CC5010E94F7367C018D
:1042600020E030E080E22F5F3F4FF701E20FF31FC5
:10427000808329303105B9F7B80121E030E0E0E072
:10428000F0E0DB014D91BD01442331F0C701820F05
:10429000931FDC014C9331962F5F3F4F2730310540
:1042A00081F7D80116968C91882369F0EE0DFF1DD9
:1042B0009DE291838A3018F4805D828304C091E38B
:1042C00092838A5D83838AE3F7018083828781E614
:1042D000838783E684878BE68587DE0112963E9688
:1042E00080E090E001962D9121938C159D05D4F3EB
:1042F000FFEF22E785E5F15020408040E1F700C064
:1043000000004091650650916606B501C7010E9404
:10431000821FC70126960FB6F894DEBF0FBECDBF31
:10432000DF91CF911F910F91FF90EF90DF90CF9091
:10433000BF90AF909F908F907F906F900C948F372D
:1043400026960FB6F894DEBF0FBECDBFDF91CF919A
:104350001F910F91FF90EF90DF90CF90BF90AF90A3
:104360009F908F907F906F9008956F927F929F9211
:10437000AF92BF92CF92DF92EF92FF920F931F9373
:10438000CF93DF931F92CDB7DEB75C018B016A013B
:104390007B0184E1E80EF11C20912C012A3098F475
:1043A00080912B018A3078F480912A018A3058F468
:1043B00080912901893038F47B01EBE1EE0EF11C8C
:1043C0009924939401C0912CC70129830E94F73648
:1043D0003C018DE3F301808380912E0181878091E0
:1043E0002D01838B88E0EAEAF6E0D3011196019073
:1043F0000D928A95E1F789E0E9EBF6E0D3011A9690
:1044000001900D928A95E1F72981911003C0C301B3
:10441000449617C080E5F301848B88E4858B87E49C
:10442000868B205D278B80912B01805D808F809112
:104430002A01805D818F80912901805D828FC30177
:104440004B960115110521F0A801B5010E945838BD
:10445000A601B701C3010E94821FC3010F90DF9123
:10446000CF911F910F91FF90EF90DF90CF90BF9071
:10447000AF909F907F906F900C948F378F929F9208
:10448000AF92BF92CF92DF92EF92FF920F931F9362
:10449000CF93DF935C016A018B016434710510F0E6
:1044A00003E410E078012FE0E20EF11CC7010E9446
:1044B000F736EC018AE3888387E090E020E030E083
:1044C0000197009769F0F901E15AF94F40814423BF
:1044D000B9F32F5F3F4FFE01E20FF31F4083F0CF90
:1044E00080912701909128018F3F4FEF940779F039
:1044F000FE01E20FF31F4DE241838A3091054CF437
:104500002E5F3F4FFE01E20FF31F805D808380E24C
:1045100009C091E392832D5F3F4FFE01E20FF31F2D
:104520008A5DF4CF293031053CF42F5F3F4FFE0107
:10453000E20FF31F8083F6CFFE01E20FF31F8AE341
:1045400081830115110581F0A801B501CE010B96FB
:104550000E945838A801B50187E696E00E945838B5
:104560001093500600934F0680911F0690912006ED
:104570000196883E23E092072CF4909320068093C6
:104580001F0604C01092200610921F06FE01E00FC5
:10459000F11F8BE7838700911F06109120069AE098
:1045A000892E912CC801B4010E948E369C0144E6EC
:1045B000A42EB12CC801B5010E948E36821B930B2C
:1045C000B4010E948E36AB01C801861B970B821B7B
:1045D000930BB5010E948E36605D6487405D458710
:1045E000205D2687A601B701CE010E94821FCE0161
:1045F000DF91CF911F910F91FF90EF90DF90CF90BF
:10460000BF90AF909F908F900C948F3720911F0692
:1046100030912006215031093093200620931F0647
:1046200060914F0670915006AC0187E696E00C94BD
:104630003E2284EF96E09F938F930E949533809162
:1046400024068F93809123068F9385E491E09F93B6
:104650008F9381EE96E09F938F930E949533809184
:1046600022068F93809121068F938FE391E09F9391
:104670008F938BEC96E09F938F930E94953380915C
:1046800038018F93809137018F9389E391E09F9355
:104690008F938BEB96E09F938F930E94953380913D
:1046A00030018F9380912F018F9381E391E09F934D
:1046B0008F938BEA96E09F938F930E9495338DB7EB
:1046C0009EB74A960FB6F8949EBF0FBE8DBF8091DD
:1046D0001E06882319F084E996E002C08CE796E074
:1046E0009F938F930E9495330F900F9080912C0190
:1046F0008A3061F01F928F9381E796E09F938F93AA
:104700000E9495330F900F900F900F9080912B0186
:104710008A3061F01F928F9385E696E09F938F9386
:104720000E9495330F900F900F900F9080912A0167
:104730008A3061F01F928F938BE596E09F938F9361
:104740000E9495330F900F900F900F908091290148
:104750008A3061F01F928F938AE496E09F938F9343
:104760000E9495330F900F900F900F9080912E0123
:104770008C3541F481E396E09F938F930E949533AB
:104780000F900F9080912E018F3241F489E196E0D5
:104790009F938F930E9495330F900F9020912D013E
:1047A000822F992787FD90959F932F938DE096E018
:1047B0009F938F930E949533809158018F9380919E
:1047C00057018F93809156018F93809155018F935C
:1047D0008CEF95E09F938F930E94953380915401C5
:1047E0008F93809153018F93809152018F93809189
:1047F00051018F938FEE95E09F938F930E94953395
:104800008DB79EB740960FB6F8949EBF0FBE8DBF72
:104810000895EF92FF920F931F93CF93DF9300D0F1
:1048200000D0CDB7DEB78C01FA01A9016115710581
:1048300009F45EC7DC018C91813209F562307105A3
:1048400008F411C761507109C80101960E94821FC6
:1048500080914B01882341F082EF9AE09F938F93E0
:104860000E9495330F900F9080914B01811140C7AA
:104870008091270681113CC78FEE9AE00AC78034E9
:10488000E9F461507109C80101960E94B521809137
:104890004B01882341F089ED9AE09F938F930E940A
:1048A00095330F900F9080914B01811121C780911A
:1048B000270681111DC786ED9AE0EBC68332E9F425
:1048C00061507109C80101960E943E2280914B01FE
:1048D000882341F088EC9AE09F938F930E94953350
:1048E0000F900F9080914B01811102C78091270694
:1048F0008111FEC685EC9AE0CCC6883419F40E947A
:104900001923F6C6833519F40E94C41EF1C68334F8
:1049100019F40E943F1DECC68C3419F40E94611DED
:10492000E7C6833609F052C06430710508F49BC6AF
:10493000E5E4F1E081E090E09C0121503109861727
:104940009707A9F08730910581F0D801A80FB91F0A
:104950002C91222331F02A3021F02D3011F02083C8
:1049600001C0108201963196E7CF26E030E0263074
:10497000310539F0F901EB5BFE4F10822F5F3F4F9D
:10498000F6CF80914B018823B1F0809124068F935C
:10499000809123068F9385E491E09F938F9382EB20
:1049A0009AE09F938F930E9495330F900F900F90F2
:1049B0000F900F900F9080914B01811199C68091BB
:1049C0002706811195C68FEA9AE063C6843609F0FE
:1049D00052C06430710508F446C6EFE3F1E081E0AF
:1049E00090E09C012150310986179707A9F0873084
:1049F000910581F0D801A80FB91F2C91222331F025
:104A00002A3021F02D3011F0208301C01082019650
:104A10003196E7CF26E030E02630310539F0F90154
:104A2000E15CFE4F10822F5F3F4FF6CF80914B012C
:104A30008823B1F0809122068F93809121068F9375
:104A40008FE391E09F938F9389E99AE09F938F93EF
:104A50000E9495330F900F900F900F900F900F9032
:104A600080914B01811144C680912706811140C677
:104A700086E99AE00EC6813309F052C062307105B2
:104A800008F4F1C5E9E3F1E081E090E09C012150F8
:104A9000310986179707A9F08730910581F0D80171
:104AA000A80FB91F2C91222331F02A3021F02D308C
:104AB00011F0208301C0108201963196E7CF26E0E5
:104AC00030E02630310539F0F901E75CFE4F108205
:104AD0002F5F3F4FF6CF80914B018823B1F080913B
:104AE00038018F93809137018F9389E391E09F93F1
:104AF0008F9386E89AE09F938F930E9495330F904F
:104B00000F900F900F900F900F9080914B0181119B
:104B1000EFC5809127068111EBC583E89AE0B9C5FE
:104B2000823309F052C06230710508F49CC5E1E39C
:104B3000F1E081E090E09C01215031098617970750
:104B4000A9F08730910581F0D801A80FB91F2C91E9
:104B5000222331F02A3021F02D3011F0208301C0C2
:104B6000108201963196E7CF26E030E026303105FD
:104B700039F0F901EF5CFE4F10822F5F3F4FF6CF07
:104B800080914B018823B1F0809130018F93809107
:104B90002F018F9381E391E09F938F9383E79AE0B6
:104BA0009F938F930E9495330F900F900F900F90CB
:104BB0000F900F9080914B0181119AC5809127062B
:104BC000811196C580E79AE064C5833709F017C163
:104BD0006330710508F447C57B01B1E0EB1AF108B9
:104BE000F8018181833609F040C0F2E0EF16F1044C
:104BF00051F0D80113968C919FEC980F993018F4CE
:104C000090E0869704C0F801828190E0C09790936D
:104C100024068093230680914B018823B1F0809174
:104C200024068F93809123068F9385E491E09F93D0
:104C30008F938DE59AE09F938F930E9495330F9009
:104C40000F900F900F900F900F9080914B0181115A
:104C50000CC080912706811108C08AE59AE09F93D5
:104C60008F930E9495330F900F90D80111968C91DD
:104C7000843609F040C0B2E0EB16F10449F0F801C7
:104C800083819FEC980F993018F490E0869705C0C7
:104C9000D80112968C9190E0C09790932206809351
:104CA000210680914B018823B1F0809122068F93D9
:104CB000809121068F938FE391E09F938F9384E4FB
:104CC0009AE09F938F930E9495330F900F900F90CF
:104CD0000F900F900F9080914B0181110CC080912B
:104CE0002706811108C081E49AE09F938F930E9468
:104CF00095330F900F90F8018181813309F03FC007
:104D000083819FEC980F9930D0F5F2E0EF16F10413
:104D100019F090E0869705C0D80112968C9190E02A
:104D2000C097909338018093370180914B0188237D
:104D3000B1F0809138018F93809137018F9389E38F
:104D400091E09F938F9381E39AE09F938F930E94CA
:104D500095330F900F900F900F900F900F908091C0
:104D60004B0181110CC080912706811108C08EE291
:104D70009AE09F938F930E9495330F900F90F801C4
:104D80008181823309F0B4C483819FEC980F9930FC
:104D900008F0AEC4F2E0EF16F10419F090E0869747
:104DA00005C0D80112968C9190E0C0979093300185
:104DB00080932F0180914B018823B1F080913001C5
:104DC0008F9380912F018F9381E391E09F938F9335
:104DD0008EE19AE09F938F930E9495330F900F90EE
:104DE0000F900F900F900F9080914B01811180C414
:104DF0008091270681117CC48BE19AE04AC48037F8
:104E000009F037C16330710508F42DC4F8018181C0
:104E10008337C9F5928180914B019133C1F491E0C0
:104E200090935001882341F088E09AE09F938F93FC
:104E30000E9495330F900F9080914B01811123C0F8
:104E40008091270681111FC085E09AE016C010925C
:104E50005001882341F081EF99E09F938F930E9446
:104E600095330F900F9080914B0181110CC0809170
:104E70002706811108C08EEE99E09F938F930E94C0
:104E800095330F900F90D80111968C91119784361D
:104E9000D1F512969C9180914B019133C1F491E030
:104EA00090934F01882341F08BED99E09F938F936E
:104EB0000E9495330F900F9080914B01811123C078
:104EC0008091270681111FC088ED99E016C01092CD
:104ED0004F01882341F084EC99E09F938F930E94C7
:104EE00095330F900F9080914B0181110CC08091F0
:104EF0002706811108C081EC99E09F938F930E944F
:104F000095330F900F90F80181818037C9F5928118
:104F100080914B019133C1F491E090934E0188232D
:104F200041F08DEA99E09F938F930E9495330F9003
:104F30000F9080914B01811123C080912706811130
:104F40001FC08AEA99E016C010924E01882341F0F2
:104F500085E999E09F938F930E9495330F900F906E
:104F600080914B0181110CC080912706811108C0EE
:104F700082E999E09F938F930E9495330F900F9051
:104F8000D80111968C9111978D36D1F512969C917E
:104F900080914B019133C1F491E090934D018823AE
:104FA00041F08EE799E09F938F930E9495330F9085
:104FB0000F9080914B01811123C0809127068111B0
:104FC0001FC08BE799E016C010924D01882341F075
:104FD00086E699E09F938F930E9495330F900F90F0
:104FE00080914B0181110CC080912706811108C06E
:104FF00083E699E09F938F930E9495330F900F90D3
:10500000F8018181893609F073C3928180914B0147
:105010009133C1F491E090934C01882341F08FE4E7
:1050200099E09F938F930E9495330F900F908091FA
:105030004B0181115DC380912706811159C38CE416
:1050400099E027C310924C01882341F087E399E04F
:105050009F938F930E9495330F900F9080914B01F7
:10506000811146C380912706811142C384E399E0F0
:1050700010C38637D1F4D80111968C91813331F465
:1050800081E080934B0189EC91E004C010924B01C8
:105090008FED91E09F938F93FF93EF930E94F40B1A
:1050A0000F900F900F900F9023C3863591F4D80185
:1050B00011968C91813341F481E080932706109200
:1050C0004B0186EF91E0E6CF109227068BE092E04D
:1050D000E1CF8C3609F041C16330710508F4C3C2D9
:1050E000F80181818C3609F05BC0615071098281C1
:1050F000813649F56A30710508F4FAC288E03396C2
:10510000AAEAB6E001900D928A95E1F780914B01F1
:10511000882371F08AEA96E09F938F938EE199E05D
:105120009F938F930E9495330F900F900F900F9045
:1051300080914B018111DCC2809127068111D8C278
:105140008BE199E0A6C28F3609F0D2C26B307105AF
:1051500008F4CEC289E0F8013396A9EBB6E00190DD
:105160000D928A95E1F780914B01882371F089EBCC
:1051700096E09F938F9383E099E09F938F930E9493
:1051800095330F900F900F900F9080914B018111EC
:10519000AFC2809127068111ABC280E099E079C24D
:1051A000803729F5828180538A3008F0A1C280932C
:1051B0002C0190914B01992379F08802C0011124B0
:1051C0009F938F938EEE98E09F938F930E949533D9
:1051D0000F900F900F900F9080914B01811188C21A
:1051E00080912706811184C28BEE98E052C28836E6
:1051F000C1F5F801828180538A3008F079C280932A
:105200002B0190914B01992309F1A1E0B0E002C07C
:10521000AA0FBB1F8A95E2F728EE33E00E947C3686
:1052200028E431E040E050E00E94C4365F934F93A1
:105230003F932F938BEC98E09F938F930E9495332D
:105240000F900F900F900F900F900F9080914B0147
:1052500081114EC28091270681114AC288EC98E0E4
:1052600018C2873631F5228120532A3008F040C217
:1052700020932A0180914B01882381F0822F992766
:1052800087FD90959F932F9386EB98E09F938F9344
:105290000E9495330F900F900F900F9080914B01CB
:1052A000811126C280912706811122C283EB98E0EA
:1052B000F0C18436D1F5F801828180538A3008F03C
:1052C00017C2893009F488E08093290180914B014D
:1052D00081110CC080912706811108C080EB98E0F5
:1052E0009F938F930E9495330F900F9080914B0165
:1052F000882309F4FDC180912901811108C087E943
:1053000098E09F938F930E9495330F900F90809118
:105310002901882309F4ECC1FDE28F9FC00111240B
:105320009F938F938DE798E013C0833709F0B8C13E
:10533000228120932D0180914B01882309F4D8C14B
:10534000822F992787FD90959F932F938BE698E066
:105350009F938F930E949533A3CE8D3609F01EC183
:105360006230710508F47FC1CB010197D801119615
:105370002C911197233609F060C0019709F4B8C148
:10538000EFE5F6E012966250710980E090E0861732
:10539000970781F08630910569F02D91222331F035
:1053A0002A3021F02D3011F0208301C010820196A7
:1053B0003196EDCF8630910531F0FC01E15AF94F7D
:1053C00010820196F7CF80914B01882359F18FE528
:1053D00096E09F938F938FE098E09F938F930E9426
:1053E000953380912701909128010F900F900F9095
:1053F0000F908F3FBFEF9B0769F09F938F938AE0D9
:1054000098E09F938F930E9495330F900F900F9089
:105410000F9008C088E098E09F938F930E94953387
:105420000F900F9080914B01811162C180912706EE
:1054300081115EC185E098E02CC1233709F05AC084
:105440008130910509F454C1029729F0F801838154
:1054500090E0869705C0D80112968C9190E0C09795
:105460009093280180932701809127019091280132
:10547000409730F08FEF9FEF9093280180932701A2
:1054800080914B01882359F18FE596E09F938F938C
:105490008DEE97E09F938F930E9495338091270123
:1054A000909128010F900F900F900F908F3FBFEFBA
:1054B0009B0769F09F938F9388EE97E09F938F935C
:1054C0000E9495330F900F900F900F9008C086EEBA
:1054D00097E09F938F930E9495330F900F90809148
:1054E0004B01811105C180912706811101C183EE15
:1054F00097E0CFC02237D1F4CA010E9406238091E1
:105500004B01882341F08DEC97E09F938F930E948D
:1055100095330F900F9080914B018111E9C08091DC
:1055200027068111E5C08AEC97E0B3C0213609F067
:10553000DFC0F801928180914B019133C1F491E079
:1055400090931E06882341F080EB97E09F938F9302
:105550000E9495330F900F9080914B018111C8C02C
:10556000809127068111C4C08DEA97E092C0109205
:105570001E06882341F082E997E09F938F930E9453
:1055800095330F900F9080914B018111B1C08091A4
:1055900027068111ADC08FE897E07BC0873761F5A2
:1055A0006230710508F45FC0AB0141505109B80188
:1055B0006F5F7F4FCE0101960E945838CE01019651
:1055C0000E941E388031F7E29F0798F4AA2797FDC2
:1055D000A095BA2F8093550190935601A09357013F
:1055E000B0935801BF93AF939F938F9389E797E050
:1055F0002CC086E597E04DC08735A9F5623071056E
:1056000090F1AB0141505109B8016F5F7F4FCE015E
:1056100001960E945838CE0101960E941E388031B2
:1056200027E29207E8F4AA2797FDA095BA2F809366
:10563000510190935201A0935301B0935401BF9331
:10564000AF939F938F9381E497E09F938F930E94F2
:1056500095330F900F900F900F900F900F9048C0C0
:105660008FE197E016C080914B01882341F087E0DD
:1056700097E09F938F930E9495330F900F908091A6
:105680004B01811135C080912706811131C084E022
:1056900097E09F938F930E9495330F900F9028C0AF
:1056A000843731F5F801928180914B01913641F4B4
:1056B0009CE590932E01882381F08AE498E007C04E
:1056C0009FE290932E01882341F08AE298E09F9315
:1056D0008F930E9495330F900F9080914B01811111
:1056E00007C080912706811103C087E298E0D1CFDF
:1056F0000F900F900F900F90DF91CF911F910F910E
:10570000FF90EF9008952F923F924F925F926F9289
:105710007F928F929F92AF92BF92CF92DF92EF9241
:10572000FF920F931F93CF93DF93CDB7DEB7C45A89
:10573000D1090FB6F894DEBF0FBECDBFC856DF4FFC
:1057400099838883C859D040C656DF4F79836883D0
:10575000CA59D040C456DF4F59834883CC59D040F2
:105760005901C257DF4F19821882CE58D0409E018E
:105770002F5F3F4FC957DF4F39832883C758D04029
:10578000AE014A575F4FC757DF4F59834883C95807
:10579000D040C856DF4F08811981C859D0400F5FEB
:1057A0001F4FC856DF4FE881F981C859D040849116
:1057B000853291F1882309F448C7C456DF4F6881C8
:1057C0007981CC59D040C656DF4FE881F981CA595A
:1057D000D0400995C257DF4FE880F980CE58D040BD
:1057E000FFEFEF1AFF0AC557DF4FB982A882CB58E7
:1057F000D040C856DF4F19830883C859D040C257DC
:10580000DF4FF982E882CE58D040C557DF4FA880DD
:10581000B980CB58D040BDCFF8018491853259F57D
:10582000C856DF4F28813981C859D0402E5F3F4F7D
:10583000C856DF4F39832883C859D040C456DF4F3C
:1058400068817981CC59D040C656DF4FE881F98113
:10585000CA59D0400995C257DF4FE880F980CE5829
:10586000D040FFEFEF1AFF0AC557DF4FB982A88279
:10587000CB58D040C4CFC256DF4F1882CE59D0404B
:10588000C357DF4F1882CD58D040C057DF4F188222
:10589000C059D040CF56DF4F1882C159D040F801CF
:1058A0002491C80101962B3209F458C060F42032CB
:1058B000E9F0233209F05AC0F1E0C357DF4FF88313
:1058C000CD58D04051C02D3251F0203309F04EC098
:1058D00021E0C256DF4F2883CE59D04045C0F1E0C9
:1058E000C057DF4FF883C059D0403EC0232D2C7FD6
:1058F000322ECF56DF4F3881C159D040332ACE5691
:10590000DF4F4881C259D04040FB32F8C057DF4FCB
:105910005881C059D04050FB33F820FA34F8CD56A6
:10592000DF4FA881C359D040A0FB35F8C357DF4FE4
:10593000B881CD58D040B0FB36F8CC56DF4FE88167
:10594000C459D040E0FB37F8232D237069F441E0BF
:10595000CF56DF4F4883C159D04006C031E0CF5603
:10596000DF4F3883C159D0408C0199CFC357DF4FE7
:105970005881CD58D040C056DF4F5883C05AD040D0
:10598000F80124912A3221F0612C712C3AE025C0D3
:1059900095012E5F3F4FD5016D907C9077FE09C039
:1059A000719461947108B1E0C057DF4FB883C0595A
:1059B000D0408C01590116C02A33A0F40F5F1F4F4D
:1059C000FC018491A301349F3001359F700C112498
:1059D00050E3651A7108680E711CC801F801249122
:1059E000203350F7C057DF4FF881C059D040FF2314
:1059F00029F0C256DF4F1882CE59D040F801849169
:105A00008E3249F5319684918A3229F08F01412CEA
:105A1000512C3AE01AC0D5014D905C900E5F1F4F9B
:105A2000F50132965F011AC02A33C0F40F5F1F4F91
:105A3000FC018491A201349F2001359F500C112458
:105A400050E3451A5108480E511CC801F801249131
:105A5000203350F703C044244A94542CF801249175
:105A6000C8010196283699F018F42C3439F017C083
:105A70002C3621F02A3799F4212C02C022242394B9
:105A80008C01CD56DF4F1882C359D0400EC08C0117
:105A9000F1E0CD56DF4FF883C359D04005C0CD5655
:105AA000DF4F1882C359D040212C98012F5F3F4F00
:105AB000C856DF4F39832883C859D040F801D490A5
:105AC000C956DF4FD882C759D040F5E6DF1609F432
:105AD00002C2FD15ECF023E5D21609F453C02D15D2
:105AE00064F035E4D31609F4F6C147E4D41609F49A
:105AF000E1C1DD2009F46FC42AC053E6D51671F167
:105B00005D150CF4C6C088E5D81609F48DC01FC019
:105B100090E7D91609F471C09D1564F0A7E6DA166E
:105B200009F4C8C1DA160CF4D1C1B9E6DB1609F4E0
:105B3000B0C00DC0E5E7DE1609F476C0F8E7DF1661
:105B400009F46DC023E7D21202C0F12C1DC0C55765
:105B5000DF4FB982A882CB58D04049C4A5014E5F1F
:105B60005F4FC557DF4F59834883CB58D040D5018D
:105B70008C918983F12C8E010E5F1F4FFE013196AF
:105B80004F0143C4FF24F39495012E5F3F4FC55747
:105B9000DF4F39832883CB58D040D5018D909C901E
:105BA0008114910421F4ADE58A2EA1E09A2E57FECE
:105BB00004C0F0E14F2EF7E25F2E8401FF20C1F018
:105BC000F8018491882309F420C4C801881999092F
:105BD000841595050CF019C40F5F1F4FF1CFC80154
:105BE00088199909841595050CF00FC40F5F1F4F94
:105BF000D8018C918111F3CF08C4F5013296C557B5
:105C0000DF4FF983E883CB58D040D5016D917C916B
:105C100080E090E0ECE7EE2EE1E0FE2E26C07CE88E
:105C2000E72E71E0F72E04C06CE7E62E61E0F62E59
:105C3000222071F0F5013496C557DF4FF983E883D0
:105C4000CB58D040D5016D917D918D919C910DC027
:105C5000C5010296F50160817181C557DF4F9983B7
:105C60008883CB58D04080E090E021E0CE56DF4FD3
:105C70002883C259D04035E7D31205C0CE56DF4F36
:105C80001882C259D040CF56DF4F1882C159D04038
:105C90003EC0222079F0A5014C5F5F4FC557DF4F12
:105CA00059834883CB58D040D5016D917D918D911A
:105CB0009C910FC0F5013296C557DF4FF983E883F9
:105CC000CB58D040D5016D917C91882777FD809588
:105CD000982F97FF13C090958095709561957F4F91
:105CE0008F4F9F4FCE56DF4F1882C259D040B2E03F
:105CF000CF56DF4FB883C159D04005C0CE56DF4FD5
:105D00001882C259D0405CE7E52E51E0F52EE1E063
:105D1000CC56DF4FE883C459D04061157105810529
:105D2000910529F4CC56DF4F1882C459D040411454
:105D3000510441F4CC56DF4FF881C459D040FF23C1
:105D400009F476C0CE56DF4F2881C259D0408E016B
:105D50000A571F4F2130A9F02AE030E040E050E020
:105D60000E94A236F701E60FF71F8081D8018E93BB
:105D70008D01B901CA01611571058105910561F7B0
:105D800015C0FB01EF70FF27EE0DFF1D2081F8010C
:105D900022938F0144E096958795779567954A956C
:105DA000D1F7611571058105910559F757FE43C07B
:105DB000C256DF4FF881CE59D040FF23E1F1232DA9
:105DC0002C7F322ECF56DF4F3881C159D040332A35
:105DD000CE56DF4F4881C259D04040FB32F8C05701
:105DE000DF4F5881C059D04050FB33F820FA34F8C7
:105DF000CD56DF4F8881C359D04080FB35F8C3575B
:105E0000DF4F9881CD58D04090FB36F8CC56DF4F0D
:105E1000A881C459D040A0FB37F8232D237081E01E
:105E200090E011F480E090E02301481A590A03C081
:105E30008E010A571F4FC757DF4F88819981C95874
:105E4000D040801B910BF80120E34F01841595058C
:105E50001CF422930196F9CFC357DF4FB881CD5878
:105E6000D040BB23A1F0CC56DF4FE881C459D040CD
:105E7000EE2369F08D2D8F7D883549F4F40131973B
:105E8000D082F2E08F1A910880E3D4018C93C95735
:105E9000DF4FE881F981C758D0408E169F0608F081
:105EA000AEC247EB52E067E17CE084E09CE00E94F8
:105EB0001734A5C2DA94DA94C956DF4FD882C7598D
:105EC000D04011E04114510469F006C0C956DF4FBB
:105ED0001882C759D04010E057FE07C026E0422E76
:105EE000512C03C044244394512C95012C5F3F4F07
:105EF000C557DF4F39832883CB58D040D501CD908B
:105F0000DD90ED90FC9020E030E0A901C701B601E2
:105F10000E94B73487FF0AC0F7FAF094F7F8F094BC
:105F2000B2E0CF56DF4FB883C159D040C156DF4FE2
:105F30001883CF59D04088248394912C8C0E9D1EB9
:105F4000860C971C20E030E040E85FE3C701B60113
:105F50000E94063687FD32C0A12CB12C27EB33E41A
:105F60004AEB51E5C701B6010E94063687FD0EC017
:105F700029EF32E045E150E5C701B6010E94BB348C
:105F80006B017C01EAE0AE0EB11CE8CF20E030E00E
:105F900040E251E4C701B6010E94063687FD49C0C0
:105FA00020E030E040E251E4C701B6010E94BB347A
:105FB0006B017C01FFEFAF1ABF0AE8CF20E030E0B1
:105FC000A901C701B6010E94B734A12CB12C8823C6
:105FD00081F12FEF36EE4BED5EE2C701B6010E9474
:105FE000B734181674F029EF32E045E150E5C701E7
:105FF000B6010E940A366B017C012AE0A21AB108A0
:10600000E8CF20E030E040E85FE3C701B6010E943E
:10601000B73487FF0EC020E030E040E251E4C70112
:10602000B6010E940A366B017C0131E0A31AB10867
:10603000E8CF112321F1A414B50464F44CEFA416A5
:106040004FEFB4063CF04A185B08C956DF4F188280
:10605000C759D04051E0451A510881E0C357DF4F7E
:106060009881CD58D0409827C156DF4F9883CF599B
:10607000D040A1E0C357DF4FA883CD58D040C956C8
:10608000DF4FB881C759D040B1114CC0B7FE3EC0F8
:1060900080E3E1E0F0E0EC0FFD1FE60DF71D8083EB
:1060A0004114510461F4C357DF4FE881CD58D0400B
:1060B000E11105C0F401319680E090E007C0F401E1
:1060C00032968EE2D40111968C93C20195012F5F16
:1060D0003F4F280F391F40E38F018217930729F0A4
:1060E000009719F041930197F7CF920120953095D1
:1060F000A216B3060CF4D6C02C01E1E0F0E0CB56BA
:10610000DF4FF983E883C559D0405CC0222733278D
:106110002A193B09CB56DF4F39832883C559D04014
:10612000840150C08401CB56DF4F19821882C559B3
:10613000D04048C0C701B6010E942335CF55DF4F7C
:10614000688379838A839B83C15AD040CF55DF4FC0
:1061500048815981C15AD040BA01882777FD80957E
:10616000982F0E9456359B01AC01C701B6010E94D1
:10617000523420E030E040E251E40E940A366B01E4
:106180007C0198012F5F3F4FCF55DF4F8881C15A67
:10619000D040805DD8018C93CB56DF4F88819981A8
:1061A000C559D0400196CB56DF4FE881F981C559DA
:1061B000D040EF2B91F0CB56DF4F99838883C559A0
:1061C000D0408901CB56DF4F28813981C559D04055
:1061D000421653060CF0AECF14C04114510439F4EA
:1061E000C357DF4FF881CD58D040FF2339F09801D5
:1061F0002E5F3F4FEEE2D8011196EC9381E090E0E4
:10620000DACF20E030E040EA50E4C701B6010E9456
:10621000063687FD47C0F80181E090E030E3229127
:106220002E3251F0820F8A3321F0808380E090E09B
:1062300003C0308381E090E08E169F0680F3892BA7
:1062400089F1C956DF4F3881C759D0403323B9F09F
:10625000F8018E169F0678F4DF018E919D018E3233
:1062600039F4CF010297DC018C918083F90101C0E0
:1062700080833197EECFBFEFAB1ABB0A0BC00F5F25
:106280001F4FF8018E169F0628F4DF018E91808340
:10629000FD01F8CF81E3E1E0F0E0EC0FFD1FE60D3A
:1062A000F71D8083C156DF4FE881CF59D040EE23E0
:1062B00049F0F8018291803311F48F01FACF8E32C8
:1062C00009F48F01C956DF4FF881C759D040FF2329
:1062D000B9F1D801FC93C8010296B7FE07C02DE2C0
:1062E00011962C93B194A194B10804C02BE2D8016B
:1062F00011962C938C01065F1F4F20E030E02F5F3A
:106300003F4FF8013196C5016AE070E00E948E3679
:10631000805DD8018C935B016115710511F08F01CF
:10632000EECF22303105DCF3E21BF30B199781919C
:106330008E932150310912161306CCF3095011091E
:10634000C256DF4FB881CE59D040BB2309F45CC0A0
:10635000E32DEC7F3E2ECF56DF4FF881C159D04060
:106360003F2ACE56DF4F2881C259D04020FB32F859
:10637000C057DF4F3881C059D04030FB33F820FA86
:1063800034F8CD56DF4F4881C359D04040FB35F833
:10639000C056DF4F5881C05AD04050FB36F8CC561B
:1063A000DF4F8881C459D04080FB37F8232D2370FC
:1063B00081E090E011F480E090E09301281B390B1C
:1063C000F40140E34F01C8018E1B9F0B8217930716
:1063D000DCF44293F7CFC557DF4FB982A882CB5880
:1063E000D040C856DF4F19830883C859D040F12CDC
:1063F0000CE511E089E5882E81E0982E06C0F12C8D
:106400008E010A571F4F01C0F12C08191909601697
:106410007106DCF1932D9C7F392ECF56DF4FA8817A
:10642000C159D0403A2ACE56DF4FB881C259D04028
:10643000B0FB32F8C057DF4FE881C059D040E0FBD5
:1064400033F820FA34F8CD56DF4FF881C359D040E5
:10645000F0FB35F8C056DF4F2881C05AD04020FBF2
:1064600036F8CC56DF4F3881C459D04030FB37F86E
:106470006301C01AD10A232D237081E090E011F44A
:1064800080E090E0C81AD90A02C0C12CD12CC057B4
:10649000DF4F4881C059D040411122C031E0C31ABA
:1064A000D108D7FC1DC0C456DF4F68817981CC5913
:1064B000D04080E2C656DF4FE881F981CA59D0400A
:1064C0000995C257DF4F28813981CE58D0402F5FC0
:1064D0003F4FC257DF4F39832883CE58D040DECF9D
:1064E000432D4C7F342ECF56DF4F5881C159D040B9
:1064F000352ACE56DF4F8881C259D04080FB32F812
:10650000C057DF4F9881C059D04090FB33F820FA34
:1065100034F8CD56DF4FA881C359D040A0FB35F8E1
:10652000C056DF4FB881C05AD040B0FB36F8CC56C9
:10653000DF4FE881C459D040E0FB37F8832D8370EA
:1065400001F1813011F48BE201C08DE2C456DF4FBE
:1065500068817981CC59D040C656DF4FE881F981F6
:10656000CA59D0400995C257DF4F28813981CE588A
:10657000D0402F5F3F4FC257DF4F39832883CE581B
:10658000D040F11009C0C257DF4FA880B980CE5863
:10659000D040A818B90822C0C257DF4FE880F98060
:1065A000CE58D0405401AE18BF080150110917FD54
:1065B0002DC0F501EE0DFF1D8491C456DF4F68819B
:1065C0007981CC59D040C656DF4FE881F981CA594C
:1065D000D0400995FFEFEF1AFF0AE7CF7501E80CED
:1065E000F91C0150110917FD11C0C456DF4F688115
:1065F0007981CC59D040D4018D914D01C656DF4FE1
:10660000E881F981CA59D0400995E8CFC057DF4FDA
:10661000F881C059D040FF2309F4F1C821E0C21A23
:10662000D108D7FCECC8C456DF4F68817981CC59BA
:10663000D04080E2C656DF4FE881F981CA59D04088
:106640000995FFEFEF1AFF0AE9CFC257DF4F8881A4
:106650009981CE58D040CC55DF4F0FB6F894DEBFAD
:106660000FBECDBFDF91CF911F910F91FF90EF90A3
:10667000DF90CF90BF90AF909F908F907F906F9062
:106680005F904F903F902F9008959091C00095FF9C
:10669000FCCF8A3041F09091C00090649093C0008C
:1066A0008093C60008959091C00090649093C000BC
:1066B0009DE09093C6009091C00095FFFCCFEBCF7A
:1066C000CF939B01C091C1004091C10048604093AD
:1066D000C1004091C1004F794093C10040E050E0BB
:1066E00065E473E30E94832B8091C00086FFFCCF9A
:1066F000C093C100CF910895CF93C091C1009091F4
:10670000C10098609093C1009091C1009F799093CF
:10671000C10060E070E00E9445338091C00086FFB8
:10672000FCCFC093C100CF910895CF93DF93CDB735
:10673000DEB7FE01359681919191BF010E946033D1
:10674000DF91CF9108951F93CF93DF931091C100F4
:106750002091C10028602093C1002091C1002F79B1
:106760002093C100FC018491EF012196882331F030
:1067700060E070E00E944533FE01F5CF8091C000DB
:1067800086FFFCCF1093C100DF91CF911F91089538
:10679000AF92BF92CF92DF92EF92FF920F931F932F
:1067A000CF93DF936C0185E0E82EF12C00E117E236
:1067B000C0E0D0E09AE0A92EB12CC601B8010E9439
:1067C0008E366C016115710529F4209719F401309A
:1067D000110529F480E3860F0E947C332196C801BD
:1067E000B5010E948E368B0181E0E81AF108E114B0
:1067F000F10419F7CE01DF91CF911F910F91FF9016
:10680000EF90DF90CF90BF90AF900895CF93DF933C
:10681000EB010E94A3338AE30E947C33CE010E94E5
:10682000C83386E49CE0DF91CF910C94A333CF93DF
:10683000DF93EC01CB01BA010E94063489E49CE0AD
:106840000E94A333CE010E94A3338AE00E947C33CE
:1068500081E090E0DF91CF9108950F931F93CF9344
:10686000DF93182F092FEB01B901CA010E940634EA
:1068700088E39CE00E94A333CE010E94A3330F93D0
:106880001F938FE29CE09F938F930E9495330F900C
:106890000F900F900F9081E090E0DF91CF911F91CA
:1068A0000F9108955058BB27AA270ED075C166D105
:1068B00030F06BD120F031F49F3F11F41EF45BC136
:1068C0000EF4E095E7FB51C1E92F77D180F3BA17B9
:1068D000620773078407950718F071F49EF58FC15E
:1068E0000EF4E0950B2EBA2FA02D0B01B9019001EB
:1068F0000C01CA01A0011124FF27591B99F0593F2F
:1069000050F4503E68F11A16F040A22F232F342F76
:106910004427585FF3CF469537952795A795F040C4
:106920005395C9F77EF41F16BA0B620B730B840BD9
:10693000BAF09150A1F0FF0FBB1F661F771F881F91
:10694000C2F70EC0BA0F621F731F841F48F48795E9
:1069500077956795B795F7959E3F08F0B3CF9395D8
:10696000880F08F09927EE0F979587950895D9D04D
:1069700008F481E008950CD00FC107D140F0FED09B
:1069800030F021F45F3F19F0F0C0511139C1F3C06C
:1069900014D198F39923C9F35523B1F3951B550BE3
:1069A000BB27AA2762177307840738F09F5F5F4FE2
:1069B000220F331F441FAA1FA9F333D00E2E3AF023
:1069C000E0E830D091505040E695001CCAF729D03D
:1069D000FE2F27D0660F771F881FBB1F261737078C
:1069E0004807AB07B0E809F0BB0B802DBF01FF27BC
:1069F00093585F4F2AF09E3F510568F0B6C000C122
:106A00005F3FECF3983EDCF3869577956795B795F5
:106A1000F7959F5FC9F7880F911D9695879597F910
:106A20000895E1E0660F771F881FBB1F6217730789
:106A30008407BA0720F0621B730B840BBA0BEE1F9E
:106A400088F7E095089504D06894B111D9C00895ED
:106A5000BCD088F09F5790F0B92F9927B751A0F07C
:106A6000D1F0660F771F881F991F1AF0BA95C9F7E2
:106A700012C0B13081F0C3D0B1E00895C0C0672F1B
:106A8000782F8827B85F39F0B93FCCF38695779592
:106A90006795B395D9F73EF490958095709561957B
:106AA0007F4F8F4F9F4F0895E89409C097FB3EF4A6
:106AB00090958095709561957F4F8F4F9F4F99234B
:106AC000A9F0F92F96E9BB279395F69587957795C9
:106AD0006795B795F111F8CFFAF4BB0F11F460FF89
:106AE0001BC06F5F7F4F8F4F9F4F16C0882311F0E1
:106AF00096E911C0772321F09EE8872F762F05C0F5
:106B0000662371F096E8862F70E060E02AF09A958F
:106B1000660F771F881FDAF7880F9695879597F984
:106B20000895990F0008550FAA0BE0E8FEEF16161E
:106B30001706E807F907C0F012161306E407F50771
:106B400098F0621B730B840B950B39F40A2661F0E5
:106B5000232B242B252B21F408950A2609F4A14088
:106B6000A6958FEF811D811D089597F99F6780E895
:106B700070E060E008959FEF80EC089500240A948F
:106B80001616170618060906089500240A94121608
:106B90001306140605060895092E0394000C11F43B
:106BA000882352F0BB0F40F4BF2B11F460FF04C0E8
:106BB0006F5F7F4F8F4F9F4F089557FD9058440F41
:106BC000551F59F05F3F71F04795880F97FB991F4C
:106BD00061F09F3F79F08795089512161306140609
:106BE000551FF2CF4695F1DF08C016161706180696
:106BF000991FF1CF86957105610508940895E89471
:106C0000BB2766277727CB0197F908958ADF08F419
:106C10008FEF08950BD0C0CFB1DF28F0B6DF18F0AA
:106C2000952309F0A2CFA7CF1124EACFC6DFA0F3A6
:106C3000959FD1F3950F50E0551F629FF001729F11
:106C4000BB27F00DB11D639FAA27F00DB11DAA1F30
:106C5000649F6627B00DA11D661F829F2227B00D7D
:106C6000A11D621F739FB00DA11D621F839FA00D08
:106C7000611D221F749F3327A00D611D231F849F58
:106C8000600D211D822F762F6A2F11249F575040AF
:106C90008AF0E1F088234AF0EE0FFF1FBB1F661F4A
:106CA000771F881F91505040A9F79E3F510570F003
:106CB0005CCFA6CF5F3FECF3983EDCF386957795EB
:106CC0006795B795F795E7959F5FC1F7FE2B880FFE
:106CD000911D9695879597F90895A29FB001B39F4E
:106CE000C001A39F700D811D1124911DB29F700DD5
:106CF000811D1124911D08950E946D36B7FF0895DE
:106D0000821B930B08950E946D36A59F900DB49F32
:106D1000900DA49F800D911D1124089597FB072EBF
:106D200016F4009407D077FD09D00E94E33607FCE3
:106D300005D03EF4909581959F4F0895709561958B
:106D40007F4F0895A1E21A2EAA1BBB1BFD010DC0A7
:106D5000AA1FBB1FEE1FFF1FA217B307E407F5070B
:106D600020F0A21BB30BE40BF50B661F771F881FE7
:106D7000991F1A9469F760957095809590959B017D
:106D8000AC01BD01CF010895052E97FB1EF40094C0
:106D90000E94DB3657FD07D00E94A23607FC03D0C5
:106DA0004EF40C94DB3650954095309521953F4F2D
:106DB0004F4F5F4F089590958095709561957F4FE7
:106DC0008F4F9F4F0895AA1BBB1B51E107C0AA1FFD
:106DD000BB1FA617B70710F0A61BB70B881F991F7C
:106DE0005A95A9F780959095BC01CD010895CF9350
:106DF000DF938230910510F482E090E0E091CB06C1
:106E0000F091CC0620E030E0A0E0B0E0309739F11E
:106E10004081518148175907B8F04817590771F454
:106E200082819381109729F013969C938E931297E9
:106E30002CC09093CC068093CB0627C0211531053A
:106E400031F04217530718F0A901DB0101C0EF012F
:106E50009A01BD01DF010280F381E02DD7CF21151A
:106E60003105F9F0281B390B2430310580F48A8173
:106E70009B816115710521F0FB019383828304C01E
:106E80009093CC068093CB06FE01329644C0FE015F
:106E9000E20FF31F819391932250310939832883A4
:106EA0003AC02091C9063091CA06232B41F42091A3
:106EB0000201309103013093CA062093C906209144
:106EC0000001309101012115310541F42DB73EB784
:106ED0004091040150910501241B350BE091C90636
:106EE000F091CA06E217F307A0F42E1B3F0B2817F8
:106EF000390778F0AC014E5F5F4F2417350748F033
:106F00004E0F5F1F5093CA064093C9068193919319
:106F100002C0E0E0F0E0CF01DF91CF910895CF9380
:106F2000DF93009709F487C0FC0132971382128225
:106F3000C091CB06D091CC06209781F4208131817D
:106F4000280F391F8091C9069091CA0682179307AE
:106F500079F5F093CA06E093C9066DC0DE0120E022
:106F600030E0AE17BF0750F412964D915C91139725
:106F70009D014115510509F1DA01F3CFB383A283D5
:106F800040815181840F951F8A179B0771F48D9161
:106F90009C911197840F951F02969183808312967E
:106FA0008D919C911397938382832115310529F448
:106FB000F093CC06E093CB063EC0D9011396FC9328
:106FC000EE9312974D915D91A40FB51FEA17FB0741
:106FD00079F480819181840F951F0296D9011196D1
:106FE0009C938E938281938113969C938E93129798
:106FF000E0E0F0E08A819B81009719F0FE01EC014E
:10700000F9CFCE01029628813981820F931F2091FA
:10701000C9063091CA062817390769F4309729F450
:107020001092CC061092CB0602C013821282D0932B
:10703000CA06C093C906DF91CF910895FC01882745
:107040009927E89421912032E9F3293010F02E306D
:10705000C8F32B3241F02D3239F4689404C00E94F9
:107060006138820F911D219120532A30C0F31EF404
:10707000909581959F4F0895911106C080538A5035
:1070800010F0865C06C0089599278827089585FD2D
:10709000FBCF80629111F8CF81568A51E0F70895B5
:1070A0009111089581568A5108F4805285580895A7
:1070B000FB01DC0102C001900D9241505040D8F715
:1070C00008957AE0979F902D879F802D910D112430
:1070D0000895DC01CB01FC01F999FECF06C0F2BD99
:1070E000E1BDF89A319600B40D9241505040B8F786
:1070F0000895F999FECF92BD81BDF89A992780B580
:107100000895A8E1B0E042E050E00C946B38DC0157
:10711000A40FB51F4150504048F0CB01840F951F7C
:107120002E910E94983841505040D0F70895262F54
:10713000F999FECF92BD81BDF89A019700B402166D
:1071400039F01FBA20BD0FB6F894FA9AF99A0FBE1B
:1071500008950196272F0E9498380C949738F89438
:02716000FFCF5F
:107162000000CD0620007001420222022000200011
:107172000064012202220200000000003F3F3F00A3
:107182003C4E554C4C3E00FFFF0A0A0A0A6E2F0283
:1071920000574944453200010057494445310041F6
:1071A200505A4D444D4E4F43414C4C010101010197
:1071B20001320000005E0100003F3F3F003C4E559F
:1071C2004C4C3E0081069806A006A106A506A20622
:1071D2004D065306600675065606A2063031323356
:1071E20034353637383941424344454630313233FB
:1071F2003435363738396162636465665352433ACF
:1072020020005B252E36732D25645D2000445354E7
:107212003A2000504154483A2000444154413A2017
:1072220000252E2A73000D0A00566572626F73657F
:10723200206D6F646520656E61626C65640A00563C
:107242006572626F7365206D6F6465206469736136
:10725200626C65640A0053696C656E74206D6F64BC
:107262006520656E61626C65640A0053696C656EC7
:1072720074206D6F64652064697361626C65640A71
:0272820000000A
:00000001FF
